:020000040000FA
:0400000007EF00F016
:1000080075829DED3EF0BAEF46F066C0D9FF67C035
:10001800DAFFDE6ADD6A68C00BF045EC42F00BC01F
:10002800B6F00CC0B7F00001B7BF0B0CD890B635CE
:10003800D96EB735DA6E8C0ED926010EDA22DECFEC
:10004800D0F0DDCFD1F0D051D11101E10C0C66C058
:10005800D9FF67C0DAFFD0C0DEFFD1C0DDFFD0C056
:10006800D9FFD1C0DAFFDF5012E020EE01F0D05105
:10007800D926D151DA22DF5023EC53F00001C26FA8
:10008800C2B105D06950D8A4C2A5000C0A0CD0C0D2
:10009800D9FFD1C0DAFFDF6A20EE01F0D051D926AE
:1000A800D151DA22B6C0DFFF20EE01F0D051D926B7
:1000B800D151DA22DF5073EC3CF00001C26FC2B1BB
:1000C800030C695002E0C2B50A0CC96BCA6BCB6B52
:1000D800CC6BD0C044F0D1C045F0466A476A486A44
:1000E800496A44EC33F00001CF6FCF0501E0D4D06A
:1000F800CD6BCE6BCE5105E1040ECD5D01E390D002
:1001080001D08ED0CDC080F0CEC081F0803B813B45
:10011800F00E811780510F0B8113F00E8017D0C09D
:1001280082F0D1C083F08051822781518323EC0E65
:100138008225C36F010E8321C46F20EE04F0C351E2
:10014800D926C451DA22DF5005E1A86BA96BAA6B46
:10015800AB6B55D020EE09F0C351D926C451DA2231
:10016800DF50816F806B20EE0AF0C351D926C4514D
:10017800DA22DF50826F82C083F0846B856B866BD6
:1001880084C086F083C085F0846B836B20EE0BF00F
:10019800C351D926C451DA22DF50876F87C088F04F
:1001A800896B8A6B8B6B88C08BF08A6B896B886BC9
:1001B800835188118C6F845189118D6F85518A11F3
:1001C8008E6F86518B118F6F80518C11906F81517A
:1001D8008D11916F000E8E11926F000E8F11936F1B
:1001E80020EE08F0C351D926C451DA22DF5090110D
:1001F800A86F9151A96F9251AA6F9351AB6FCD51CE
:10020800040DF350980FD96EDA6AA8C0DEFFA9C0B2
:10021800DEFFAAC0DEFFABC0DEFFCD4BCE2B6AD718
:10022800CD6BCE6BCD51CE1103E0CD07D8A0CE0754
:10023800CD51040DF350980FD96EDA6ADECFC9F0AC
:10024800DECFCAF0DECFCBF0DECFCCF0C951CA1179
:10025800CB11CC1105E1000EAD6F020EAC6F11D0C1
:10026800D0C044F0D1C045F0C9C046F0CAC047F07C
:10027800CBC048F0CCC049F044EC33F00001AC6F7F
:10028800AD6BACC0CFF0CF5107E0CD4BCE2BCE51EC
:1002980003E1040ECD5DCCE3030ECF1901E1010C9F
:1002A800CF5101E00D0C20EE3AF0D051D926D151B2
:1002B800DA22DF50816F806B20EE39F0D051D926D9
:1002C800D151DA22DF508013020E8119801101E02A
:1002D8000D0C20EE45F0D051D926D151DA22DF504D
:1002E800816F806B20EE44F0D051D926D151DA22AB
:1002F800DF50801380C0C5F081C0C6F0C76BC86BE3
:10030800C551C611C711C81155E120EE53F0D0519F
:10031800D926D151DA22DF50816F806B20EE54F05C
:10032800D051D926D151DA22DF50826F82C083F0B2
:10033800846B856B866B84C086F083C085F0846B84
:10034800836B20EE55F0D051D926D151DA22DF50F7
:10035800876F87C088F0896B8A6B8B6B88C08BF03E
:100368008A6B896B886B835188118C6F84518911D2
:100378008D6F85518A118E6F86518B118F6F8051C9
:100388008C11906F81518D11916F000E8E11926FAB
:10039800000E8F11936F20EE52F0D051D926D15113
:1003A800DA22DF509011C56F9151C66F9251C76F15
:1003B8009351C86F20EE16F0D051D926D151DA22C8
:1003C800C5C0DEFFC6C0DEFFC7C0DEFFC8C0DEFF97
:1003D80020EE3EF0D051D926D151DA2210EE03F0AA
:1003E800D051E126D151E222DFCFE7FF20EE03F022
:1003F800D051D926D151DA22DE040AE020EE03F0EA
:10040800D051D926D151DA22020EDE1801E00D0CA6
:10041800C5C00BF0C6C00CF0C7C00DF0C8C00EF0C8
:1004280020EE03F0D051D926D151DA22DF500F6ED9
:10043800106A116A126A41EC4BF00BC0C5F00CC08F
:10044800C6F00DC0C7F00EC0C8F020EE3BF0D0518A
:10045800D926D151DA2210EE02F0D051E126D1513D
:10046800E222DFCFE7FF20EE02F0D051D926D151AA
:10047800DA22DF50D8B40D0C20EE02F0D051D92684
:10048800D151DA22DF50806F20EE02F0D051D92608
:10049800D151DA22DF50816F8105801501E00D0C02
:1004A80020EE40F0D051D926D151DA22DF50816FA9
:1004B800806B20EE3FF0D051D926D151DA22DF509F
:1004C800801320EE08F0D051D926D151DA2280C00D
:1004D800DEFF81C0DDFF20EE08F0D051D926D151D2
:1004E800DA22DF50806F0F0E801701E00D0C20EE2E
:1004F80042F0D051D926D151DA22DF50816F806B7A
:1005080020EE41F0D051D926D151DA22DF508013A4
:1005180080C0BAF081C0BBF0BC6BBD6BBA51BB11D7
:10052800BC11BD1155E120EE4FF0D051D926D15163
:10053800DA22DF50816F806B20EE50F0D051D9263F
:10054800D151DA22DF50826F82C083F0846B856BD1
:10055800866B84C086F083C085F0846B836B20EE45
:1005680051F0D051D926D151DA22DF50876F87C098
:1005780088F0896B8A6B8B6B88C08BF08A6B896B70
:10058800886B835188118C6F845189118D6F8551C7
:100598008A118E6F86518B118F6F80518C11906FDD
:1005A80081518D11916F000E8E11926F000E8F1177
:1005B800936F20EE4EF0D051D926D151DA22DF5078
:1005C8009011BA6F9151BB6F9251BC6F9351BD6F2F
:1005D80020EE3CF0D051D926D151DA22DF50806F7D
:1005E80020EE3DF0D051D926D151DA22DF50816F6B
:1005F8008051B86F81C0B9F0B851B91101E10D0C43
:1006080020EE08F0D051D926D151DA22DECF80F081
:10061800DDCF81F0040E826FD89081338033822F32
:10062800FBD7B8518025836FB9518121846F856BC1
:10063800D8B0852B866BC5518325B26FC6518421EE
:10064800B36FC7518521B46FC8518621B56FB251B8
:10065800BA5DB351BB59B451BC59B551BD5901E24A
:100668000D0CB251BA5D0B6EB351BB590C6EB4513F
:10067800BC590D6EB551BD590E6E20EE02F0D05129
:10068800D926D151DA22DF500F6E106A116A126A28
:10069800C1EC4BF00BC0BEF00CC0BFF00DC0C0F0F9
:1006A8000EC0C1F00001BE51BF11C011C11101E15E
:1006B8000D0C010ECF6FC151C01105E1F60EBE5DE4
:1006C8000F0EBF5902E3020ECF6FC151C01105E1F1
:1006D800F60EBE5DFF0EBF5902E3030ECF6F020E8A
:1006E800BE25806F000EBF21816F000EC021826F72
:1006F800000EC121836F20EE12F0D051D926D151BE
:10070800DA2280C0DEFF81C0DEFF82C0DEFF83C048
:10071800DEFF20EE1AF0D051D926D151DA22C9C015
:10072800DEFFCAC0DEFFCBC0DEFFCCC0DEFFB851A3
:10073800C925806FB951CA21816F000ECB21826F04
:10074800000ECC21836F20EE1EF0D051D926D15156
:10075800DA2280C0DEFF81C0DEFF82C0DEFF83C0F8
:10076800DEFFB251C925806FB351CA21816FB451E0
:10077800CB21826FB551CC21836F20EE26F0D0516A
:10078800D926D151DA2280C0DEFF81C0DEFF82C0C7
:10079800DEFF83C0DEFF030ECF1901E08CD020EE10
:1007A80008F0D051D926D151DA22DE50DE1001E00E
:1007B8000D0C20EE5BF0D051D926D151DA22DF5052
:1007C800816F806B20EE5CF0D051D926D151DA22AE
:1007D800DF50826F82C083F0846B856B866B84C028
:1007E80086F083C085F0846B836B20EE5DF0D0517A
:1007F800D926D151DA22DF50876F87C088F0896BFC
:100808008A6B8B6B88C08BF08A6B896B886B835182
:1008180088118C6F845189118D6F85518A118E6F63
:1008280086518B118F6F80518C11906F81518D1172
:10083800916F000E8E11926F000E8F11936F20EE44
:100848005AF0D051D926D151DA22DF509011946F45
:100858009151956F9251966F9351976F20EE22F0B8
:10086800D051D926D151DA2294C0DEFF95C0DEFFDF
:1008780096C0DEFF97C0DEFF20EE12F0D051D926D9
:10088800D151DA22DECF80F0DECF81F0DECF82F0E8
:10089800DECF83F0020ED8908037813782378337D6
:1008A800E82EF9D780C0AEF081C0AFF082C0B0F0BA
:1008B80083C0B1F0B7D020EE08F0D051D926D1517D
:1008C800DA22DE50DE1001E10D0C20EE1EF0D051D0
:1008D800D926D151DA22DECF80F0DECF81F0DECF0B
:1008E80082F0DECF83F0C5518025846FC651812107
:1008F800856FC7518221866FC8518321876F20EE8B
:1009080022F0D051D926D151DA2284C0DEFF85C029
:10091800DEFF86C0DEFF87C0DEFF020ECF196BE068
:1009280020EE12F0D051D926D151DA22DECF80F054
:10093800DECF81F0DECF82F0DECF83F0010E8015AE
:10094800846F856B866B876B20EE12F0D051D926A9
:10095800D151DA22DECF88F0DECF89F0DECF8AF0FF
:10096800DECF8BF0030E8803F3CF8CF0F4CF8DF03D
:100978008E6B8F6B8903F3508D27F4508E23000EF6
:100988008F238803F3508D27F4508E23000E8F2376
:10099800030E8A03F3508E27F4508F23000E890329
:1009A800F3508E27F4508F23000E8803F3508E27C0
:1009B800F4508F23030E8B03F3508F27000E8A0306
:1009C800F3508F27000E8903F3508F27000E8803FA
:1009D800F3508F27D8908F338E338D338C338451D7
:1009E8008C25AE6F85518D21AF6F86518E21B06FEA
:1009F80087518F2116D020EE12F0D051D926D1512F
:100A0800DA22DECF80F0DECF81F0DECF82F0DECFDB
:100A180083F0D8908035AE6F8135AF6F8235B06F77
:100A28008335B16FFF0EAE25806F010EAF21816F48
:100A3800000EB021826F000EB121836F0A0E05D01F
:100A4800D8908333823381338033E82EF9D720EE70
:100A580016F0D051D926D151DA228051DE5C81516D
:100A6800DE588251DE588351DE5801E20D0C20EE2B
:100A78000EF0D051D926D151DA22DE68DE68DE6860
:100A8800DD68DD52DD5210EE0AF0D051E126D15179
:100A9800E222DECFE6FFDECFE6FFDECFE6FFDECFE7
:100AA800E6FF20EE05F0D051D926D151DA22800E8A
:100AB800DF6E030ECF1901E0D3D120EE5FF0D051E5
:100AC800D926D151DA22DF50816F806B20EE5EF09B
:100AD800D051D926D151DA22DF50801380058111F7
:100AE80001E0BED1D0C039F0D1C03AF0C9293B6E7F
:100AF800000ECA213C6E000ECB213D6E000ECC21AB
:100B08003E6EFEEC48F0000901E0AAD1000120EE9B
:100B180005F0D051D926D151DA22DF6A22EE2DF024
:100B2800D051D926D151DA22DF50816F806B22EE65
:100B38002CF0D051D926D151DA22DF508013550E2E
:100B4800801903E1AA0E8119D8A48AD120EE2FF0CA
:100B5800D051D926D151DA22DF50816F806B20EE37
:100B680030F0D051D926D151DA22DF50826F82C0BD
:100B780083F0846B856B866B84C086F083C085F0B8
:100B8800846B836B20EE31F0D051D926D151DA2213
:100B9800DF50876F87C088F0896B8A6B8B6B88C042
:100BA8008BF08A6B896B886B835188118C6F8451A9
:100BB80089118D6F85518A118E6F86518B118F6FB8
:100BC80080518C11906F81518D11916F000E8E1193
:100BD800926F000E8F11936F20EE2EF0D051D92610
:100BE800D151DA22DF509011946F9151956F925143
:100BF800966F9351976F520E941909E1520E9519F9
:100C080006E1610E961903E1410E9719D8A428D17F
:100C180022EE13F0D051D926D151DA22DF50816F5C
:100C2800806B22EE14F0D051D926D151DA22DF5050
:100C3800826F82C083F0846B856B866B84C086F07C
:100C480083C085F0846B836B22EE15F0D051D926D2
:100C5800D151DA22DF50876F87C088F0896B8A6BA1
:100C68008B6B88C08BF08A6B896B886B835188117A
:100C78008C6F845189118D6F85518A118E6F8651C1
:100C88008B118F6F80518C11906F81518D11916FE5
:100C9800000E8E11926F000E8F11936F22EE12F0DC
:100CA800D051D926D151DA22DF509011946F915149
:100CB800956F9251966F9351976F720E941909E13F
:100CC800720E951906E1410E961903E1610E971906
:100CD800D8A4C6D022EE17F0D051D926D151DA22A5
:100CE800DF50816F806B22EE18F0D051D926D15198
:100CF800DA22DF50826F82C083F0846B856B866B4B
:100D080084C086F083C085F0846B836B22EE19F073
:100D1800D051D926D151DA22DF50876F87C088F0A9
:100D2800896B8A6B8B6B88C08BF08A6B896B886B3D
:100D3800835188118C6F845189118D6F85518A1167
:100D48008E6F86518B118F6F80518C11906F8151EE
:100D58008D11916F000E8E11926F000E8F11936F8F
:100D680022EE16F0D051D926D151DA22DF50901157
:100D7800946F9151956F9251966F9351976F20EEA2
:100D88000EF0D051D926D151DA2294C0DEFF95C099
:100D9800DEFF96C0DEFF97C0DEFF22EE1BF0D051CB
:100DA800D926D151DA22DF50816F806B22EE1CF0F8
:100DB800D051D926D151DA22DF50826F82C083F018
:100DC800846B856B866B84C086F083C085F0846BEA
:100DD800836B22EE1DF0D051D926D151DA22DF5093
:100DE800876F87C088F0896B8A6B8B6B88C08BF0A4
:100DF8008A6B896B886B835188118C6F8451891138
:100E08008D6F85518A118E6F86518B118F6F80512E
:100E18008C11906F81518D11916F000E8E11926F10
:100E2800000E8F11936F22EE1AF0D051D926D151AE
:100E3800DA22DF509011946F9151956F9251966F0D
:100E48009351976F20EE0AF0D051D926D151DA226A
:100E580094C0DEFF95C0DEFF96C0DEFF97C0DEFFC0
:100E6800D0C0D9FFD1C0DAFFCFC0DFFF01018A4B64
:100E78008B2B000120EE06F0D051D926D151DA2271
:100E88008AC1DEFF8BC1DDFF000C0C6A0B6AC7EC60
:100E980052F00F0B0101FB6F976B070E966E010E58
:100EA800FC6FA06B0F0EC16E926893689468948E65
:100EB800929092928982020EFA6F18EC52F09294F4
:100EC800898492988998929E899E95689368460E1F
:100ED8000001806FFB0E816FA70E826FFF0E836F7C
:100EE800EC0E846FFE0E856F2E0E866FFF0E876FD9
:100EF800DDEC52F0AEEC52F017D0B90E0001806F65
:100F0800FE0E816F82CF82F0836BDDEC52F0150EFE
:100F18000001F96F4B0EF86FBE0EE82EFED7F82FC2
:100F2800FCD7F92FFAD700F082B2E7D7E6EC43F006
:100F38000101FB6F660E0001806FFC0E816FFBC123
:100F480082F0836BDDEC52F00400150E0001F96F9E
:100F58004B0EF86FBE0EE82EFED7F82FFCD7F92FF0
:100F6800FAD700F0F286F180F288F19CF28E7AECE2
:100F78004EF0899289944DEC46F04DEC46F0000E07
:100F88000B6E340E99EC4FF0490E0F6EFF0E106E7B
:100F980084EC4BF0A70E0F6EFF0E106E84EC4BF036
:100FA800000E0B6E390E99EC4FF089800400D2ECDC
:100FB8002FF0EBEC3DF0FCEC4BF0000E0B6E800ECE
:100FC80099EC4FF00101FB510F0D340EF3240F6E15
:100FD8000C0EF420106E84EC4BF00101965101E1E7
:100FE800EAD0A70E0001806FFD0E816FDDEC52F094
:100FF8006FEC4CF00FC0D9F110C0DAF111C0DBF181
:1010080012C0DCF10101D951DA11DB11DC1117E151
:10101800AD0E0001806FFC0E816FD9C182F0DAC17C
:1010280083F0DBC184F0DCC185F0DDEC52F00A0E00
:101038000E6E000E0F6A106A116AF8EC4EF001018C
:10104800DD6BDE6BDEBF05D0DE5119E1040EDD5D20
:1010580016E2DC0E0001806FFF0E816FD90E0101D0
:10106800DD25D96E010EDE21DA6EDF500001826FB8
:10107800836BDDEC52F00101DD4BDE2BE3D7730E01
:101088000001806FFB0E816FDDEC52F0330E000122
:10109800806FFC0E816FDDEC52F022EE00F000EE66
:1010A800CAF01F0EDBCFEBFFE806FCE2D40E00010E
:1010B800EA6FFF0EEB6F0DEC31F0CAC078F1CBC0D0
:1010C80079F1CCC07AF1CDC07BF101017851791169
:1010D8007A117B1170E0190E0001806FFC0E816F90
:1010E80078C182F079C183F07AC184F07BC185F040
:1010F800DDEC52F0000E0001A36F020EA46F78C160
:10110800F9F079C1FAF07AC1FBF0F86B000EF82516
:10111800A56F010EF921A66F000EFA21A76F000E28
:10112800FB21A86F63EC0EF0000E626E020E636E78
:10113800340E646E0A0E656E676A080E666ED70E08
:10114800686E010E696E4DEC11F00101DF6BE06B0A
:10115800E0BF05D0E05119E1080EDF5D16E2D80EB8
:101168000001806FFF0E816F340E0101DF25D96EFB
:101178000A0EE021DA6EDF500001826F836BDDEC2E
:1011880052F00101DF4BE02BE3D72AEE34F0DF50B9
:10119800CE6FCF6BD06BD16B8F0E0001806FFE0EC0
:1011A800816FCEC182F0CFC183F0D0C184F0D1C1AC
:1011B80085F0DDEC52F00101A0AF13D0946889925C
:1011C8008982150E0001F96F4B0EF86FBE0EE82EDE
:1011D800FED7F82FFCD7F92FFAD700F044EC37F0F8
:1011E800EED7FC510CE0C70E0001806FFD0E816F39
:1011F800DDEC52F0020E01019B6F220E0BD0B70EF0
:101208000001806FFD0E816FDDEC52F0010E0101CF
:101218009B6F040E9A6FD36BD46BE46B899E000EA0
:10122800E36F010EE26FE3BF05D0E35162E1040E04
:10123800E25D5FE20F0EE203F3CFF8F0F4CFF9F0CE
:10124800E303F3500001F927240EF8250B6E0D0E69
:10125800F9210C6E21EC50F00C5003E1030E0B5CED
:1012680044E3170E0001806FFE0E816F0F0E01011F
:10127800E203F3CFF8F0F4CFF9F0E303F350000101
:10128800F927240EF825826F0D0EF921836FDDEC06
:1012980052F0E2C1F8F0E3C1F9F0050ED890000170
:1012A800F837F937E82EFAD7000EF825D26F020E74
:1012B800F921D36F0F0E0101E203F3CFFAF0F4CF57
:1012C800FBF0E303F3500001FB27240EFA25D46F4B
:1012D8000D0EFB21D56F030ED66F68EC16F00101D9
:1012E800D56FD66BD55121EC4FF00101E24BE32BC2
:1012F8009AD7899E000E0B6EC00E99EC4FF055ECF4
:1013080052F0000E0B6EC00E99EC4FF0950E0F6E5A
:10131800FF0E106E84EC4BF0FAD081A8939429EC60
:1013280053F00B500C1001E1D3D0E4C1D2F1E10E1F
:101338000B6E010E0C6EB8EC4AF00101E46F350E2D
:10134800E41907E1730E0001806FFB0E816FDDEC7D
:1013580052F0370E0001806FFF0E816FE4C182F0FA
:10136800836B010E80A0000E846F856BDDEC52F05C
:101378000101E1A91DD0600EE4191AE15F0ED2192E
:1013880017E1FA832AEE34F09BC1DFFF2AEE35F02D
:101398009AC1DFFF8984496A020E486E56EC35F01F
:1013A8008994FA93726A86EC52F00101E46BAFD02B
:1013B800FC5143E0E151100B0001A66F000EA76F2E
:1013C8000101E45131EC38F0A6C0E5F1A7C0E6F11F
:1013D800080E0101E519E61101E100F0070E01010F
:1013E800E519E61102E168EC4DF0E505E61102E1C8
:1013F800D5EC4CF0020EE519E61102E104EC3AF0E6
:10140800030EE519E61106E15AEC2AF0E1C0D3F122
:10141800E2C0D4F1050E0101E519E61106E14EEC32
:1014280036F0EAC0D3F1EBC0D4F1090E0101E51999
:10143800E6116DE11DEC53F06AD0E151100B0B6E13
:10144800000E0C6EE45120EC25F00BC0E5F10CC049
:10145800E6F1070E0101E519E61102E1A3EC4CF0F3
:10146800020EE519E61102E173EC4FF0E505E6110D
:1014780002E1E5EC3FF0030EE519E61102E142EC6A
:1014880050F0040EE519E61102E1AAEC51F0050E40
:10149800E519E61102E1D7EC42F0060E0101E51963
:1014A800E61102E132EC53F0080EE519E61102E10B
:1014B800E9EC3AF0090EE519E61102E1E9EC44F02D
:1014C8000A0E0101E519E61122E162EC45F01FD090
:1014D800E6EC43F00101976F985119E0FB51971919
:1014E80016E0898E000E0B6EC00E99EC4FF055EC8D
:1014F80052F0000E0B6EC00E99EC4FF0040E0F6EFA
:10150800FF0E106E84EC4BF097C1FBF132D082B223
:1015180030D0050E0101D319D4112BE0FED6B90E37
:101528000001806FFE0E816F82CF82F0836BDDEC4D
:1015380052F0150E0001F96F4B0EF86FBE0EE82E33
:10154800FED7F82FFCD7F92FFAD700F00400000EC9
:101558000B6EC00E99EC4FF055EC52F0000E0B6E6E
:10156800C00E99EC4FF0510E0F6EFF0E106E84EC0A
:101578004BF082B2D4D7150E0001F96F4B0EF86FFD
:10158800BE0EE82EFED7F82FFCD7F92FFAD700F0B9
:10159800000E23EC53F00101956FF20E0001806FED
:1015A800FC0E816F95C182F0836BDDEC52F0150E55
:1015B8000001F96F4B0EF86FBE0EE82EFED7F82F1C
:1015C800FCD7F92FFAD700F0899489920001D26BE1
:1015D800D36B750ED46FFB0ED56FD66B4CEC49F000
:1015E800E5D4A5C0B7F0A6C0B8F0A951D96EDA6A9B
:1015F800DE6ADD6AA3C00CF0A4C00DF071EC4AF0FD
:101608000001B66FB65102E0B651120020EE05F0A7
:10161800A351D926A451DA22DF5008E020EE05F0C4
:10162800A351D926A451DA22DF50120020EE04F08B
:10163800A351D926A451DA22DFA2070C20EE06F026
:10164800A351D926A451DA2210EE06F0A351E126BF
:10165800A451E222E6CFAEF0E6CFAFF0E6CFB0F08D
:10166800E6CFB1F0A751AE25B26FA851AF21B36F45
:10167800000EB021B46F000EB121B56FDE50B25D1F
:10168800DE50B359DE50B459DE50B55901E3E1D20A
:10169800A76BA86BDED220EE06F0A351D926A45181
:1016A800DA22FF0EDE14AA6F010EDE14AB6F000EF5
:1016B800DE14AC6F000EDE14AD6FAA51AB11AC1185
:1016C800AD1101E032D220EE06F0A351D926A45183
:1016D800DA22DECFAAF0DECFABF0DECFACF0DECF81
:1016E800ADF00A0E05D0D890AD33AC33AB33AA3386
:1016F800E82EF9D7A3C0D9FFA4C0DAFF10EE02F094
:10170800DE50E126DD50E222E750AE6FAE05AA15A5
:10171800B96FB95101E099D020EE06F0A351D9264E
:10172800A451DA22DE50DE10DE10DE1022E120EEB7
:101738000EF0A351D926A451DA22DECFC0F0DECFB5
:10174800C1F0DECFC2F0DECFC3F0C051C111C2116B
:10175800C3112FE1A3C0D9FFA4C0DAFFDECF8CF0FC
:10176800DDCF8DF08E6B8F6B906B916B28EC2DF02D
:1017780018D0A3C0D9FFA4C0DAFFDECF8CF0DDCF2C
:101788008DF020EE12F0A351D926A451DA22DECF33
:101798008EF0DECF8FF0DECF90F0DECF91F028EC28
:1017A8002DF08CC0C0F08DC0C1F08EC0C2F08FC0CB
:1017B800C3F0C051C111C211C31101E14ED2C0051D
:1017C800C111C211C31109E120EE05F0A351D926B8
:1017D800A451DA22020EDF6E020CC0290FE1C129E2
:1017E8000DE1C2290BE1C32909E120EE05F0A3515F
:1017F800D926A451DA22010EDF6E010C20EE12F078
:10180800A351D926A451DA22C0C0DEFFC1C0DEFF31
:10181800C2C0DEFFC3C0DEFF20EE0EF0A351D92602
:10182800A451DA22DE50DE10DE10DE100EE120EECA
:101838000EF0A351D926A451DA22C0C0DEFFC1C0E0
:10184800DEFFC2C0DEFFC3C0DEFF20EE16F0A351EC
:10185800D926A451DA22A3C0E1FFA4C0E2FF00EE1A
:101868002AF0E650E926E550EA22DE50EE1816E1A5
:10187800DE50EE1813E1DE50EE1810E1DE50EE18DF
:101888000DE1A3C0D9FFA4C0DAFFDECF24F0DDCF7D
:1018980025F042EC3FF0000901E083D1A3C0D9FF55
:1018A800A4C0DAFFDECF0BF0DDCF0CF0000120EE94
:1018B80012F0A351D926A451DA22DECF0DF0DECFE3
:1018C8000EF0DECF0FF0DECF10F05FEC43F00BC070
:1018D800BCF00CC0BDF00DC0BEF00EC0BFF00001E2
:1018E800BC51BD11BE11BF1101E16ED7B951BC2762
:1018F800000EBD23BE23BF23A7C0AAF0A8C0ABF02B
:10190800090EAC6FD890AB33AA33AC2FFBD7AAC063
:10191800BAF0ABC0BBF0BA51BB1101E1C3D0B951A9
:10192800BA25AA6F000EBB21AB6FA3C0D9FFA4C014
:10193800DAFF10EE02F0DE50E126DD50E222E75039
:10194800AC6FAD6BAA51AC5DAB51AD5912E2A3C0FF
:10195800D9FFA4C0DAFF10EE02F0DE50E126DD5018
:10196800E222E750AA6FB951AA5DBA6FBB6BD8A043
:10197800BB07B7C01AF0B8C01BF0BCC01CF0BDC094
:101988001DF0BEC01EF0BFC01FF0BAC020F0BBC023
:1019980021F0A3C0D9FFA4C0DAFF10EE01F0DE5099
:1019A800E126DD50E222E750DBEC45F0000901E0DA
:1019B800F8D00001BA51AA6FBB51AB6FAC6BAD6BDD
:1019C800A3C0D9FFA4C0DAFF10EE2AF0DE50E1264A
:1019D800DD50E222E6CFAEF0E6CFAFF0E6CFB0F0D2
:1019E800E6CFB1F0BC51AE5DB26FBD51AF59B36F28
:1019F800BE51B059B46FBF51B159B56FAA51B25D5C
:101A0800AB51B359AC51B459AD51B5593CE2A3C02F
:101A1800D9FFA4C0DAFFDECFAAF0DDCFABF02E0EDF
:101A2800AA250B6E000EAB210C6EA3C0D9FFA4C073
:101A3800DAFF10EE2AF0DE50E126DD50E222E6CF92
:101A4800ACF0E5CFADF0BC51AC5FBD51AD5B090E5C
:101A5800D890AC37AD37E82EFBD7AC51B7250D6E13
:101A6800AD51B8210E6E020E106E0F6A62EC50F086
:101A7800A3C0D9FFA4C0DAFF10EE04F0DE50E126BF
:101A8800DD50E222E76ABAC0AAF0BBC0ABF0090E8B
:101A9800D890AA37AB37E82EFBD7AAC0C4F0ABC0A2
:101AA800C5F0BBD020EE0AF0A351D926A451DA2202
:101AB80010EE06F0A351E126A451E222DE50E65CC6
:101AC800DE50E658DE50E658DE50E6581FE3A3C065
:101AD800D9FFA4C0DAFFDECF24F0DDCF25F042EC39
:101AE8003FF0000901E05DD0A3C0D9FFA4C0DAFF30
:101AF80010EE2AF0DE50E126DD50E222BCC0E6FFFF
:101B0800BDC0E6FFBEC0E6FFBFC0E6FF000120EE95
:101B180016F0A351D926A451DA22BCC0DEFFBDC0FD
:101B2800DEFFBEC0DEFFBFC0DEFFAA69010EAB6FDD
:101B380020EE06F0A351D926A451DA22DECFACF06C
:101B4800DDCFADF0AA51AC17AB51AD17AC510008C1
:101B5800C46FAD51D8A0E82A0208C56FC451A75D6B
:101B6800C551A85904E2A7C0C4F0A8C0C5F0A3C0D5
:101B7800D9FFA4C0DAFFDECF39F0DDCF3AF020EE8E
:101B880016F0A351D926A451DA22DECF3BF0DECFDE
:101B98003CF0DECF3DF0DECF3EF0FEEC48F0000931
:101BA80002E0000122D60001AA69010EAB6F20EE07
:101BB80006F0A351D926A451DA22DECFACF0DDCF4E
:101BC800ADF0AA51AC17AB51AD17A3C0D9FFA4C053
:101BD800DAFFDECFAEF0DDCFAFF0AC51AE27AD51BE
:101BE800AF232E0EAE250B6E000EAF210C6EB7C0C4
:101BF8000DF0B8C00EF0C4C00FF0C5C010F062EC14
:101C080050F0A3C0D9FFA4C0DAFF10EE04F0DE50F4
:101C1800E126DD50E222010EE76EC451B727C55117
:101C2800B82320EE06F0A351D926A451DA22C451D4
:101C3800DE26C551DE22000EDE22DE22A951D96E33
:101C4800DA6AC451DE26C551DD22C451A75FC551E9
:101C5800A85BA751A81101E01ED520EE06F0A351FC
:101C6800D926A451DA2210EE0AF0A351E126A45194
:101C7800E222DE50E65CDE50E658DE50E658DE50E2
:101C8800E65814E220EE06F0A351D926A451DA2230
:101C980010EE0AF0A351E126A451E222DECFE6FFBE
:101CA800DECFE6FFDECFE6FFDECFE6FF20EE04F074
:101CB800A351D926A451DA22000EDB8A000CA3C056
:101CC8000CF0A4C00DF071EC4AF00001BD6FBD51DD
:101CD80002E0BD51120020EE05F0A351D926A4510F
:101CE800DA22DF5008E020EE05F0A351D926A451EE
:101CF800DA22DF50120020EE0AF0A351D926A451AF
:101D0800DA22A551DE5CA651DE58A751DE58A8514B
:101D1800DE5816E220EE04F0A351D926A451DA22A7
:101D2800DFB20ED020EE0AF0A351D926A451DA2250
:101D3800DECFA5F0DECFA6F0DECFA7F0DECFA8F08D
:101D480020EE06F0A351D926A451DA22DECFB9F04D
:101D5800DECFBAF0DECFBBF0DECFBCF0BE6BBF6B20
:101D6800C06BC16B20EE06F0A351D926A451DA222C
:101D7800BEC0DEFFBFC0DEFFC0C0DEFFC1C0DEFFE9
:101D8800A551A611A711A81101E119D2A3C0D9FF25
:101D9800A4C0DAFF10EE02F0DE50E126DD50E222A8
:101DA800E750A96FA9C0AAF0AB6BAC6BAD6B090E7D
:101DB800D890AA37AB37AC37AD37E82EF9D7AAC0D9
:101DC800C2F0ABC0C3F0ACC0C4F0ADC0C5F0B951EF
:101DD800BA11BB11BC1101E196D0FF0EA5250B6EFF
:101DE800FF0EA6210C6EFF0EA7210D6EFF0EA82177
:101DF8000E6EC2C00FF0C3C010F0C4C011F0C5C051
:101E080012F0C1EC4BF00BC0A9F00CC0AAF00DC049
:101E1800ABF00EC0ACF0FF0E0001B9250B6EFF0E43
:101E2800BA210C6EFF0EBB210D6EFF0EBC210E6E8B
:101E3800C2C00FF0C3C010F0C4C011F0C5C012F08A
:101E4800C1EC4BF00B500001A95D0C50AA590D5084
:101E5800AB590E50AC5957E3FF0EC225A96FFF0EC0
:101E6800C321AA6FFF0EC421AB6FFF0EC521AC6F53
:101E7800A91DAD6FAA1DAE6FAB1DAF6FAC1DB06FC6
:101E8800FF0EB925B16FFF0EBA21B26FFF0EBB214D
:101E9800B36FFF0EBC21B46FAD51B115B56FAE5124
:101EA800B215B66FAF51B315B76FB051B415B86F5F
:101EB80020EE06F0A351D926A451DA22B5C0DEFFE0
:101EC800B6C0DEFFB7C0DEFFB8C0DEFF20EE06F00A
:101ED800A351D926A451DA22DE50A55FDE50A65BB5
:101EE800DE50A75BDD50A85B20EE12F0A351D92687
:101EF800A451DA22DECFC6F0DECFC7F0DECFC8F0BD
:101F0800DECFC9F064D020EE0EF0A351D926A4513B
:101F1800DA22DECFC6F0DECFC7F0DECFC8F0DECFE4
:101F2800C9F0C651C711C811C91143E1A3C0D9FFEF
:101F3800A4C0DAFFDECF8CF0DDCF8DF08E6B8F6B17
:101F4800906B916B28EC2DF08CC0C6F08DC0C7F05B
:101F58008EC0C8F08FC0C9F0C605C711C811C91115
:101F680009E120EE05F0A351D926A451DA22020E88
:101F7800DF6E020CC6290FE1C7290DE1C8290BE164
:101F8800C92909E120EE05F0A351D926A451DA2286
:101F9800010EDF6E010C20EE0EF0A351D926A451DC
:101FA800DA22C6C0DEFFC7C0DEFFC8C0DEFFC9C078
:101FB800DEFF20EE12F0A351D926A451DA22C6C0C2
:101FC800DEFFC7C0DEFFC8C0DEFFC9C0DEFFC651E6
:101FD800C711C811C91101E095D0F1D020EE04F065
:101FE800A351D926A451DA22DFA228D0A3C0D9FF51
:101FF800A4C0DAFFDECF8CF0DDCF8DF0C6C08EF046
:10200800C7C08FF0C8C090F0C9C091F028EC2DF07F
:102018008CC0C6F08DC0C7F08EC0C8F08FC0C9F0A4
:10202800C651C711C811C91123E1C2C0A5F0C3C068
:10203800A6F0C4C0A7F0C5C0A8F06ED0A3C0D9FF51
:10204800A4C0DAFFDECF44F0DDCF45F0C6C046F0CD
:10205800C7C047F0C8C048F0C9C049F028EC1BF019
:1020680044C0C6F045C0C7F046C0C8F047C0C9F074
:102078000001C62907E1C72905E1C82903E1C929E3
:1020880001E180D7C951C811C71104E1020EC65D2C
:1020980001E267D7A3C0D9FFA4C0DAFF10EE12F09F
:1020A800DE50E126DD50E222E650C65DE650C75913
:1020B800E650C859E650C95901E353D720EE12F04B
:1020C800A351D926A451DA22C6C0DEFFC7C0DEFF5D
:1020D800C8C0DEFFC9C0DEFF20EE06F0A351D92636
:1020E800A451DA22C251DE26C351DE22C451DE22B7
:1020F800C551DE22C251A55FC351A65BC451A75B7F
:10210800C551A85BA551C25DA651C359A751C45971
:10211800A851C55901E262D720EE06F0A351D9268D
:10212800A451DA22A551DE26A651DE22A751DE22CD
:10213800A851DE22A551A96F010EA615AA6FAB6B97
:10214800AC6BA911AB11AC113AE0A3C0D9FFA4C084
:10215800DAFFDECF0BF0DDCF0CF0C6C00DF0C7C044
:102168000EF0C8C00FF0C9C010F05FEC43F00BC010
:10217800BEF00CC0BFF00DC0C0F00EC0C1F0000131
:10218800BE51BF11C011C11101E1EBD6A5C0A9F024
:10219800A6C0AAF0A7C0ABF0A8C0ACF00A0E05D044
:1021A800D890AC33AB33AA33A933E82EF9D7A95169
:1021B800BE27AA51BF23AB51C023AC51C12320EE87
:1021C80006F0A351D926A451DA22FF0EDE14A96F16
:1021D800010EDE14AA6F000EDE14AB6F000EDE14C3
:1021E800AC6FA951AA11AB11AC1120E020EE16F08A
:1021F800A351D926A451DA22BE51DE1809E1BF51F4
:10220800DE1806E1C051DE1803E1C151DE180EE008
:1022180020EE16F0A351D926A451DA22BEC0DEFF63
:10222800BFC0DEFFC0C0DEFFC1C0DEFF20EE06F08B
:10223800A351D926A451DA2210EE0AF0A351E126BF
:10224800A451E222DE50E65CDE50E658DE50E65845
:10225800DE50E65801E33DD520EE06F0A351D9261D
:10226800A451DA2210EE0AF0A351E126A451E22289
:10227800DECFE6FFDECFE6FFDECFE6FFDECFE6FF0E
:1022880020EE04F0A351D926A451DA22000EDB8AED
:1022980020D564C0A1F065C0A2F068C0D9FF69C0AC
:1022A800DAFFDE6ADD6A62C00CF063C00DF071EC23
:1022B8004AF000019C6F9C5102E09C51120020EEF4
:1022C80005F06250D9266350DA22DF5008E020EE8C
:1022D80005F06250D9266350DA22DF50120020EE52
:1022E80004F06250D9266350DA22DFA0070C20EEF2
:1022F80006F06250D9266350DA22DECF8CF0DECFAA
:102308008DF0DECF8EF0DECF8FF020EE0AF0625037
:10231800D9266350DA22DECF90F0DECF91F0DECFFF
:1023280092F0DECF93F08C51905D986F8D5191595A
:10233800996F8E5192599A6F8F5193599B6F66502E
:102348008C6F67508D6F8E6B8F6B8C51985D8D5134
:1023580099598E519A598F519B5901E34AD298C085
:1023680066F099C067F045D220EE06F06250D92693
:102378006350DA22FF0EDE148C6F010EDE148D6FAF
:10238800000EDE148E6F000EDE148F6F8C518D11CF
:102398008E118F1101E0A5D120EE06F06250D926EA
:1023A8006350DA22DECF8CF0DECF8DF0DECF8EF0F8
:1023B800DECF8FF00A0E05D0D8908F338E338D3351
:1023C8008C33E82EF9D762C0D9FF63C0DAFF10EE6C
:1023D80002F0DE50E126DD50E222E750906F9005D2
:1023E8008C15A36FA3516AE120EE06F06250D9263E
:1023F8006350DA22DE50DE10DE10DE100FE120EE30
:102408000EF06250D9266350DA22DECF9DF0DECF7F
:102418009EF0DECF9FF0DECFA0F020D062C0D9FFC3
:1024280063C0DAFFDECF44F0DDCF45F020EE12F0D6
:102438006250D9266350DA22DECF46F0DECF47F06D
:10244800DECF48F0DECF49F028EC1BF044C09DF009
:1024580045C09EF046C09FF047C0A0F00001A051C3
:102468009F119E110CE1020E9D5D09E220EE05F020
:102478006250D9266350DA22020EDF6E020C9D29C3
:102488000FE19E290DE19F290BE1A02909E120EE2A
:1024980005F06250D9266350DA22010EDF6E010C76
:1024A80020EE12F06250D9266350DA229DC0DEFF7A
:1024B8009EC0DEFF9FC0DEFFA0C0DEFF62C0D9FF66
:1024C80063C0DAFFDECF0BF0DDCF0CF020EE12F0A8
:1024D8006250D9266350DA22DECF0DF0DECF0EF03F
:1024E800DECF0FF0DECF10F05FEC43F00BC0A4F0AE
:1024F8000CC0A5F00DC0A6F00EC0A7F00001A451B5
:10250800A511A611A71101E1B1D7A351A427000E67
:10251800A523A623A72366C08CF067C08DF0090EFB
:102528008E6FD8908D338C338E2FFBD78CC0A8F04C
:102538008DC0A9F0A851A91101E1C5D0A351A825C2
:102548008C6F000EA9218D6F62C0D9FF63C0DAFFBE
:1025580010EE02F0DE50E126DD50E222E7508E6FE9
:102568008F6B8C518E5D8D518F5912E262C0D9FFED
:1025780063C0DAFF10EE02F0DE50E126DD50E22201
:10258800E7508C6FA3518C5DA86FA96BD8A0A907E1
:10259800A1C01AF0A2C01BF0A4C01CF0A5C01DF079
:1025A800A6C01EF0A7C01FF0A8C020F0A9C021F047
:1025B80062C0D9FF63C0DAFF10EE01F0DE50E126F9
:1025C800DD50E222E750ACEC48F0000901E05FD7AB
:1025D80062C0D9FF63C0DAFF10EE04F0DE50E126D6
:1025E800DD50E222E7505FE00001A8518C6FA9514D
:1025F8008D6F8E6B8F6B62C0D9FF63C0DAFF10EEF0
:102608002AF0DE50E126DD50E222E6CF90F0E6CF58
:1026180091F0E6CF92F0E6CF93F0A451905D946FDD
:10262800A5519159956FA6519259966FA7519359F3
:10263800976F8C51945D8D5195598E5196598F5144
:10264800975931E262C0D9FF63C0DAFF10EE2AF071
:10265800DE50E126DD50E222E6CF8CF0E5CF8DF0AA
:10266800A4518C5FA5518D5B090ED8908C378D379E
:10267800E82EFBD78C51A1250B6E8D51A2210C6E33
:1026880062C0D9FF63C0DAFFDECF8EF0DDCF8FF0F6
:102698002E0E8E250D6E000E8F210E6E020E106E00
:1026A8000F6A62EC50F0A8C08CF0A9C08DF0090E3A
:1026B800D89000018C378D37E82EFAD78CC0AAF055
:1026C8008DC0ABF079D020EE16F06250D926635059
:1026D800DA22A4C0DEFFA5C0DEFFA6C0DEFFA7C0C9
:1026E800DEFF8C69010E8D6F20EE06F06250D92650
:1026F8006350DA22DECF8EF0DDCF8FF08C518E174B
:102708008D518F178E510008AA6F8F51D8A0E82AD3
:102718000208AB6FAA51665CAB51675804E266C009
:10272800AAF067C0ABF062C0D9FF63C0DAFFDECFA2
:1027380039F0DDCF3AF020EE16F06250D92663501A
:10274800DA22DECF3BF0DECF3CF0DECF3DF0DECF4D
:102758003EF0FEEC48F0000901E099D6A1C00BF06C
:10276800A2C00CF000018C69010E8D6F20EE06F0FE
:102778006250D9266350DA22DECF8EF0DDCF8FF09B
:102788008C518E178D518F1762C0D9FF63C0DAFF45
:10279800DECF90F0DDCF91F08E5190278F519123AD
:1027A8002E0E90250D6E000E91210E6EAAC00FF010
:1027B800ABC010F062EC50F0AA51A127AB51A22394
:1027C80020EE06F06250D9266350DA22AA51DE269E
:1027D800AB51DE22000EDE22DE2268C0D9FF69C0BE
:1027E800DAFFAA51DE26AB51DD22AA51665EAB5153
:1027F800675A6650671001E0B7D5000C276E266A45
:1028080001D227500AE10001FC5107E0266A0101C4
:10281800856B0A0E86D0899055D2020E271808E1DA
:102828000001FC5105E0266A0101856B140E79D080
:102838001F0E276430D0300E27602DD00001FC51C8
:102848002AE02750E00F736E266A7350200D0A0E97
:10285800F324D96E020EF420DA6EDE50DE10DE109C
:10286800DE1003E0030E73642BD0010E6B6E735001
:10287800140D130EF324D96E010EF420DA6E735082
:10288800140D130EF324E16E010EF420E26EE750EE
:102898000409DF6E15D03F0E276416D0500E27604E
:1028A80013D00001FC5110E07350140D000EF324F6
:1028B800D96E010EF420DA6E2750C00FDF6E266A3B
:1028C8000101846B856BA7D7340E271808E1000136
:1028D800FC5105E00101846B856B266A9CD7350E97
:1028E800271809E10001FC5106E0266A0D0E0101D6
:1028F800856FAC0E16D0370E271808E10001FC5181
:1029080005E00E0E0101856F750E74D10D0E2718A6
:102918000AE10001FC5107E0266A020E0101856FF9
:10292800BC0E846F78D7100E271808E10001FC51FF
:1029380005E0030E0101856FE90E5CD1180E27181A
:1029480008E10001FC5105E0070E0101856F090E41
:1029580051D13E0E271801E0B5D10001FC5101E12B
:10296800B1D10F0E0101856F3D0E44D17350140D86
:10297800010EF324D96E010EF420DA6E27C0DFFFB2
:10298800030E0101856FEA0E35D17350140D020E46
:10299800F324D96E010EF420DA6E27C0DFFF030E90
:1029A8000101856FEB0E26D17350140D030EF3242D
:1029B800D96E010EF420DA6E27C0DFFF030E010185
:1029C800856FEC0E17D17350140D040EF324D96ED5
:1029D800010EF420DA6E27C0DFFF030E0101856FB8
:1029E800ED0E08D17350140D050EF324D96E010EA7
:1029F800F420DA6E27C0DFFF030E0101856FEE0EAB
:102A0800F9D07350140D060EF324D96E010EF4207C
:102A1800DA6E27C0DFFF7350140D060EF324D96E4B
:102A2800010EF420DA6EDF500B6E0BC00CF00D6A4D
:102A38000E6A0F6A0EC00FF00DC00EF00CC00DF03C
:102A48000C6A7350140D050EF324D96E010EF42090
:102A5800DA6EDF50106E10C011F0126A136A146A31
:102A680012C014F011C013F0126A116A7350140DD9
:102A7800040EF324D96E010EF420DA6EDF50156EC1
:102A880015C016F0176A186A196A16C019F0186A7C
:102A9800176A166A7350140D030EF324D96E010ECB
:102AA800F420DA6EDF5016241A6E000E17201B6E03
:102AB800000E18201C6E000E19201D6E11501A24CD
:102AC8001E6E12501B201F6E13501C20206E1450B7
:102AD8001D20216E0C501E24226E0D501F20236EC7
:102AE8000E502020246E0F502120256E7350140D97
:102AF800070EF324D96E010EF420DA6E22C0DEFF31
:102B080023C0DEFF24C0DEFF25C0DEFF6BD073507C
:102B1800140D120EF324D96E010EF420DA6E27C0BC
:102B2800DFFF070E0101856F0A0E64D07350140D84
:102B3800110EF324D96E010EF420DA6E27C0DFFFE0
:102B4800070E0101856F0B0E55D07350140D100E32
:102B5800F324D96E010EF420DA6E27C0DFFF070ECA
:102B68000101856F0C0E46D07350140D0F0EF3241F
:102B7800D96E010EF420DA6E27C0DFFF33D027C0EC
:102B88006CF10F0E0101856F3E0E34D027C06DF138
:102B98000F0E0101856F3F0E2DD027C06EF10F0E6D
:102BA8000101856F400E26D027C06FF10F0E01017D
:102BB800856F410E1FD027C070F10F0E0101856F80
:102BC800420E18D027C071F10F0E0101856F430E18
:102BD80011D027C072F10F0E0101856F440E0AD083
:102BE80027C073F10101846B856B6CD00E0E010157
:102BF800856F760E846F66D00101846B856B090E34
:102C0800266E09D684C10BF085C10CF00C500FE07C
:102C1800030A11E0040A23E00A0A2FE0030A32E05B
:102C2800010A36E0130A49E03B0A4AE04BD00B5050
:102C380001E1E7D547D00B50E90A01E197D6030A2D
:102C480001E1A3D6010A01E1AFD6070A01E1BBD62B
:102C5800010A01E1C7D6030A01E1D3D633D00B50EC
:102C6800090A01E154D7030A01E160D7010A01E129
:102C78006CD7070A01E178D725D00B50480AB2E093
:102C8800E40A20D00B50750AB1E0030AB5E01AD067
:102C98000B503D0A01E173D7030A01E177D7010A16
:102CA80001E17BD77F0A80E0010A85E0030A8AE018
:102CB800010A8FE0070A94E005D00B502A0A02D0D7
:102CC8000B500F0A26501200D251D31101E1090C02
:102CD800D2C0D9FFD3C0DAFFDE6ADD6A8CC1B8F191
:102CE8008DC1B9F11F0ED617B80E666E010E676E4C
:102CF800D40E686ED651FE0B696E09EC00F0010126
:102D0800B56FB55101E040D2A10ECC6F010ECD6F69
:102D1800B80E0001BC6F010EBD6FD4C0BEF0D5C0A7
:102D2800BFF031EC3DF00101B56FCAC1B6F1CBC1BE
:102D3800B7F1B55105E1B651B71102E1060EB56F0D
:102D4800D6C0D7F01C0E0001D71701E114D101013C
:102D5800B55113E0040EB51909E1B80E0001C06FB2
:102D6800010EC16FF6EC47F00101B56F0001D6877F
:102D7800CAC1B6F1CBC1B7F113D020EE0BF0B651F2
:102D8800D926B751DA22DF500001D76F110ED717B5
:102D980002E0070E03D0D6A503D0080E0101B56FD7
:102DA8000101B55101E002D10001D6A7FFD0010110
:102DB800B16BB26B210EB36F460EB46F20EE0EF0FE
:102DC800B651D926B751DA22DF6A20EE0FF0B65194
:102DD800D926B751DA22B2C1DFFF20EE10F0B65182
:102DE800D926B751DA22B3C1DFFF20EE11F0B65170
:102DF800D926B751DA22B4C1DFFF20EE16F0B6515A
:102E0800D926B751DA22DF6A20EE17F0B651D92653
:102E1800B751DA22B2C1DFFF20EE18F0B651D92639
:102E2800B751DA22B3C1DFFF20EE19F0B651D92627
:102E3800B751DA22B4C1DFFF20EE0BF0B651D92624
:102E4800B751DA22DF6A20EE1CF0B651D926B75105
:102E5800DA22DF6A20EE1DF0B651D926B751DA2200
:102E6800DF6A20EE1EF0B651D926B751DA22DF6AA2
:102E780020EE1FF0B651D926B751DA22DF6AB8C161
:102E88000BF0B9C10CF0B6C10DF0B7C10EF057EC9C
:102E980048F00BC0ADF10CC0AEF10DC0AFF10EC0E3
:102EA800B0F1B6C10BF0B7C10CF00D6A0E6A0F6A2B
:102EB800106A00EC50F0010120EE04F0B851D92658
:102EC800B951DA22010EDF6EAD51AE11AF11B0115A
:102ED8006DE020EE2AF0B851D926B951DA22DECFBA
:102EE800B1F1DECFB2F1DECFB3F1DECFB4F1B8C1CC
:102EF8008CF0B9C18DF0ADC18EF0AEC18FF0AFC10D
:102F080090F0B0C191F0AFEC41F00101B56FB5514F
:102F18004DE1FF0EAD250001D76FFF0E0101AE2177
:102F28000001D86FFF0E0101AF210001D96FFF0E1C
:102F38000101B0210001DA6F010120EE0AF0B85159
:102F4800D926B951DA22D7C0DEFFD8C0DEFFD9C0F2
:102F5800DEFFDAC0DEFFB8C139F0B9C13AF0B1C15D
:102F68003BF0B2C13CF0B3C13DF0B4C13EF0FEEC61
:102F780048F001011AD00101B55118E120EE0BF01B
:102F8800B651D926B751DA22DFA802D0040E0DD0E7
:102F98000001D6A30BD0010120EE0BF0B651D926C3
:102FA800B751DA22DFA002D0070EB56F0101B55183
:102FB80023E10001D6B7D68B010120EE2AF0B851E3
:102FC800D926B951DA22000110EE1AF0D251E126C1
:102FD800D351E222DECFE6FFDECFE6FFDECFE6FF0B
:102FE800DECFE6FF20EE1EF0D251D926D351DA22E9
:102FF800B6C1DEFFB7C1DDFF0101B55101E0C4D0A4
:10300800000120EE04F0D251D926D351DA22D6C0DD
:10301800DFFF20EE05F0D251D926D351DA22DF6A3C
:10302800B8C10BF0B9C10CF0B6C10DF0B7C10EF0C4
:1030380057EC48F0000120EE0EF0D251D926D351BA
:10304800DA220BC0DEFF0CC0DEFF0DC0DEFF0EC0B3
:10305800DEFF010120EE1DF0B651D926B751DA2264
:10306800DF500001D86FD76B010120EE1EF0B6517A
:10307800D926B751DA22DF500001D96FD9C0DAF06A
:10308800DB6BDC6BDD6BDBC0DDF0DAC0DCF0DB6B4F
:10309800DA6B010120EE1FF0B651D926B751DA22BA
:1030A800DF500001DE6FDEC0DFF0E06BE16BE26B4A
:1030B800DFC0E2F0E16BE06BDF6BDA51DF11E36F49
:1030C800DB51E011E46FDC51E111E56FDD51E211F4
:1030D800E66FD751E311E76FD851E411E86F000E9E
:1030E800E511E96F000EE611EA6F010120EE1CF010
:1030F800B651D926B751DA22DF500001E711EB6F3C
:10310800E851EC6FE951ED6FEA51EE6F20EE0AF0ED
:10311800D251D926D351DA22EBC0DEFFECC0DEFF54
:10312800EDC0DEFFEEC0DEFF20EE06F0D251D9265C
:10313800D351DA22DE6ADE6ADE6ADD6A20EE16F034
:10314800D251D926D351DA22DE6ADE6ADE6ADD6A16
:10315800D2C0D9FFD3C0DAFFB8C1DEFFB9C1DDFFE5
:10316800D2C0D9FFD3C0DAFF10EE06F0DE50E12658
:10317800DD50E22220EE02F0D251D926D351DA22D4
:10318800E6CFDEFFE5CFDDFF0101B5511200495062
:103198004810471003E1020E465C10E320EE12F0DF
:1031A8004450D9264550DA22DE50465CDE50475856
:1031B800DE504858DE50495801E22FD2020E866F81
:1031C80041D246C084F047C085F0D89085314F6E13
:1031D80084314E6E4E5084274F50852344C039F0B9
:1031E80045C03AF020EE1EF04450D9264550DA2268
:1031F800DECF4EF0DECF4FF0DECF50F0DECF51F015
:1032080084C052F085C053F0090E546ED8905332E2
:103218005232542EFBD752504E243B6E53504F20FF
:103228003C6E000E50203D6E000E51203E6EFEECAE
:1032380048F00001866F865101E004D24E68010E05
:103248004F6E84C050F085C051F04E5050164F500C
:10325800511644C052F045C053F0505052265150B8
:1032680053222E0E5224876F000E5320886F844BF2
:10327800852B46B004D04AC080F0816B1AD04A50E2
:103288004E6E4F6A4E3A4F3AF00E4F164E500F0B95
:103298004F12F00E4E1687C0D9FF88C0DAFFDF50F4
:1032A8000F0B506E516A4E505010806F4F50511096
:1032B800816F87C0D9FF88C0DAFF80C0DFFF20EEAA
:1032C80004F04450D9264550DA22010EDF6E44C07E
:1032D80039F045C03AF020EE1EF04450D92645504A
:1032E800DA22DECF4EF0DECF4FF0DECF50F0DECF69
:1032F80051F084C052F085C053F0090E546ED89036
:1033080053325232542EFBD752504E243B6E5350F8
:103318004F203C6E000E50203D6E000E51203E6E38
:10332800FEEC48F00001866F865101E08BD14E68B3
:10333800010E4F6E84C050F085C051F04E505016AB
:103348004F50511644C052F045C053F050505226C9
:10335800515053222E0E5224876F000E5320886F2F
:1033680046B00CD04BC04EF00F0E4E1687C0D9FF9A
:1033780088C0DAFFDF50F00B4E1012D04AC04EF072
:103388004BC04FF04CC050F04DC051F0050E05D069
:10339800D890513250324F324E32E82EF9D74E5033
:1033A800826F836B87C0D9FF88C0DAFF82C0DFFFD6
:1033B8002BD144C039F045C03AF020EE1EF04450FD
:1033C800D9264550DA22DECF4EF0DECF4FF0DECFE1
:1033D80050F0DECF51F04750526E4850536E49506E
:1033E800546E556A4E5052243B6E4F5053203C6EDB
:1033F800505054203D6E515055203E6EFEEC48F022
:103408000001866F865101E01DD14E68010E4F6E96
:1034180046C050F047C051F0D890503651364E5003
:1034280050164F50511644C052F045C053F05050FA
:103438005226515053222E0E5224876F000E5320CD
:10344800886F87C0D9FF88C0DAFF4AC0DFFF20EE47
:1034580001F08751D9268851DA224BC0DFFFD4D03A
:1034680044C039F045C03AF020EE1EF04450D92649
:103478004550DA22DECF4EF0DECF4FF0DECF50F0EF
:10348800DECF51F046C052F047C053F048C054F068
:1034980049C055F0080E05D0D890553254325332F1
:1034A8005232E82EF9D74E5052243B6E4F505320DB
:1034B8003C6E505054203D6E515055203E6EFEECEF
:1034C80048F00001866F865101E0BCD04E68010EBD
:1034D8004F6E46C050F047C051F0D8905036513624
:1034E800D890503651364E5050164F50511644C051
:1034F80052F045C053F050505226515053222E0ED0
:103508005224876F000E5320886F20EE01F08751F8
:10351800D9268851DA22DF504F6E4E6A20EE02F02B
:103528008751D9268851DA22DF50506E50C051F0A9
:10353800526A536A546A52C054F051C053F0526AE6
:10354800516A20EE03F08751D9268851DA22DF50DC
:10355800556E55C056F0576A586A596A56C059F0A0
:10356800586A576A566A515056105A6E5250571038
:103578005B6E535058105C6E545059105D6E4E502F
:103588005A105E6E4F505B105F6E000E5C10606EDE
:10359800000E5D10616E87C0D9FF88C0DAFFDF506A
:1035A8005E10626E5F50636E6050646E6150656E4F
:1035B800666A676A686AF00E6514696E66504A1230
:1035C80067504B1268504C1269504D1287C0D9FF92
:1035D80088C0DAFF4AC0DFFF20EE01F08751D92604
:1035E8008851DA224BC0DFFF20EE02F08751D9263E
:1035F8008851DA224CC0DFFF20EE03F08751D9262C
:103608008851DA224DC0DFFF20EE04F04450D9265D
:103618004550DA22010EDF6E15D044C0D9FF45C0EF
:10362800DAFFDF504E6E4F6A4F5001E0C7D54E505B
:10363800010A01E1C6D5030A01E1BBD6010A01E18D
:103648000FD7BCD58651120049504810471003E1E6
:10365800020E465C0FE320EE12F04450D926455086
:10366800DA22DE50465CDE504758DE504858DE50BD
:10367800495808E3010E0001846F000E856B866BC4
:10368800876BEFD100018469856986698769D4D120
:1036980046C088F047C089F0D89089314B6E883190
:1036A8004A6E4A5088274B50892344C039F045C098
:1036B8003AF020EE1EF04450D9264550DA22DECFEB
:1036C8004AF0DECF4BF0DECF4CF0DECF4DF088C0B5
:1036D8004EF089C04FF0090E506ED8904F324E32DE
:1036E800502EFBD74E504A243B6E4F504B203C6E19
:1036F800000E4C203D6E000E4D203E6EFEEC48F054
:10370800000901E0AED14A68010E4B6E88C04CF04A
:1037180089C04DF04A504C164B504D1644C04EF0DF
:1037280045C04FF04C504E264D504F222E0E4E2481
:10373800D96E000E4F20DA6EDF500001826F836B66
:10374800884B892B44C039F045C03AF020EE1EF072
:103758004450D9264550DA22DECF4AF0DECF4BF06E
:10376800DECF4CF0DECF4DF088C04EF089C04FF070
:10377800090E506ED8904F324E32502EFBD74E5015
:103788004A243B6E4F504B203C6E000E4C203D6E41
:10379800000E4D203E6EFEEC48F0000901E061D1BC
:1037A8004A68010E4B6E88C04CF089C04DF04A50F3
:1037B8004C164B504D1644C04EF045C04FF04C507F
:1037C8004E264D504F222E0E4E24D96E000E4F20FD
:1037D800DA6EDF50516E506A50500001821351501A
:1037E800831346B006D08251806F0F0E8315816F08
:1037F8000FD082C04AF083C04BF0040E4C6ED890B4
:103808004B324A324C2EFBD74AC080F04BC081F075
:1038180080C084F081C085F05BD044C039F045C0D9
:103828003AF020EE1EF04450D9264550DA22DECF79
:103838004AF0DECF4BF0DECF4CF0DECF4DF04750F4
:103848004E6E48504F6E4950506E516A4A504E2441
:103858003B6E4B504F203C6E4C5050203D6E4D50AF
:1038680051203E6EFEEC48F0000901E0FAD04A68AB
:10387800010E4B6E46C04CF047C04DF0D8904C3608
:103888004D364A504C164B504D1644C04EF045C06C
:103898004FF04C504E264D504F222E0E4E24000114
:1038A8008A6F000E4F208B6F20EE01F08A51D926C7
:1038B8008B51DA22DF504B6E4A6A8AC0D9FF8BC01F
:1038C800DAFFDF504A12000E4AC084F04BC085F080
:1038D800866B876BC6D044C039F045C03AF020EEFD
:1038E8001EF04450D9264550DA22DECF4AF0DECF0A
:1038F8004BF0DECF4CF0DECF4DF046C04EF047C067
:103908004FF048C050F049C051F0080E05D0D8908B
:10391800513250324F324E32E82EF9D74A504E24A7
:103928003B6E4B504F203C6E4C5050203D6E4D50DE
:1039380051203E6EFEEC48F0000901E092D04A6842
:10394800010E4B6E46C04CF047C04DF0D8904C3637
:103958004D36D8904C364D364A504C164B504D1675
:1039680044C04EF045C04FF04C504E264D504F22AB
:103978002E0E4E2400018A6F000E4F208B6F20EE12
:1039880001F08A51D9268B51DA22DF504B6E4A6AF0
:1039980020EE02F08A51D9268B51DA22DF504C6E84
:1039A8004CC04DF04E6A4F6A506A4EC050F04DC040
:1039B8004FF04E6A4D6A20EE03F08A51D9268B519A
:1039C800DA22DF50516E51C052F0536A546A556A78
:1039D80052C055F0546A536A526A4D505210566E8E
:1039E8004E505310576E4F505410586E505055103B
:1039F800596E4A5056105A6E4B5057105B6E000E57
:103A080058105C6E000E59105D6E8AC0D9FF8BC0CD
:103A1800DAFFDF505A105E6E5B505F6E5C50606E6E
:103A28005D50616E5E50846F5F50856F6050866F29
:103A38000F0E6114876F15D044C0D9FF45C0DAFF57
:103A4800DF504A6E4B6A4B5001E014D64A50010AC7
:103A580001E11ED6030A01E1E0D6010A01E13BD7E4
:103A680009D684C044F085C045F086C046F087C0BA
:103A780047F012002A6E1BC041F01CC042F02A50C9
:103A880001E0040C010E3F6E74B0030CE9D1BBECED
:103A980052F0000901E1FDD13F6AFBD1146A156AB1
:103AA800166A176A090E12EC51F0000901E0F1D10B
:103AB8002B0E0B6E0C6A0E6A100E0D6E4EEC4EF04D
:103AC800000901E1E6D12B44E846030BE8064DE185
:103AD80032C01DF03F0E1D161DC01EF01F6A206A61
:103AE800216A1FC021F01EC020F01F6A1E6A3350D1
:103AF800236E226A3450246E256A225024262350CD
:103B0800252224501E24266E25501F20276E000EC5
:103B18002020286E000E2120296E26283B6E000EDC
:103B280027203C6E000E28203D6E000E29203E6E98
:103B38003BC01DF03CC01EF03DC01FF03EC020F051
:103B48000A0ED8901D361E361F362036E82EF9D7B5
:103B58001BC0D9FF1CC0DAFF1DC0DEFF1EC0DEFF80
:103B68001FC0DEFF20C0DEFF97D71D6A35AE01D02B
:103B78001D2A010E1D1630C01EF00F0E1E163450E1
:103B8800030B020DF3501E241D24020F406E31500A
:103B9800030B1D6E1E6A0A0ED8901D361E36E82EBF
:103BA800FBD732501F6E206AD8901F362036D89027
:103BB8001F3620363344E846030B216E226A1F5015
:103BC8002126205022221D5021261E502222212A41
:103BD800000E222221C03BF022C03CF03D6A3E6A22
:103BE80040C01DF0F70E1D263BC01EF03CC01FF064
:103BF8003DC020F03EC021F01D2A05D0D8901E36C9
:103C08001F36203621361D2EF9D734D06EA43FD06A
:103C1800146A156A166A176A8D0E12EC51F00009BB
:103C280001E037D116EC53F02B0E0B6E0C6A0E6ABE
:103C3800100E0D6E4EEC4EF0000901E12AD1300E47
:103C4800406E03D016EC53F040064050FBE135C0FF
:103C58001DF01D3A0F0E1D16100E1E6E1F6A206AEB
:103C6800216A1D2A05D0D8901E361F3620362136E7
:103C78001D2EF9D71BC0D9FF1CC0DAFF1EC0DEFFFE
:103C88001FC0DEFF20C0DEFF21C0DEFF05D7146A9B
:103C9800156A166A176A090E12EC51F0000901E05C
:103CA800F8D02B0E0B6E0C6A0E6A100E0D6E4EECD1
:103CB8004EF0000901E1EDD06EA232D038C01DF0FF
:103CC800060E1E6ED8901D321E2EFCD7FF0E1D2626
:103CD80035503F0B1F6E206AD8901F362036364469
:103CE800010B1F26000E20221F2A20221D2A03D086
:103CF800D8901F3620361D2EFBD71F50216E20501E
:103D0800226E236A246A1BC0D9FF1CC0DAFF21C0B7
:103D1800DEFF22C0DEFF23C0DEFF24C0DEFFBCD6EC
:103D28003650030B1D6E1E6AD8901D361E36D8906D
:103D38001D361E36D8901D361E363638E842070B1B
:103D48001D26000E1E221D2A1E223540E8423F0B6A
:103D58001F0B1F6E206A1F2A000E20221D501F02F3
:103D6800F3CF21F0F4CF22F02002F35022261E5088
:103D78001F02F35022262150236E2250246E256AFA
:103D8800266A1BC0D9FF1CC0DAFF23C0DEFF24C08F
:103D9800DEFF25C0DEFF26C0DEFF7ED641C0D9FF8C
:103DA80042C0DAFF6EC0DFFF77D6146A156A166A5A
:103DB800176A090E12EC51F000096BE141C00BF0D3
:103DC80042C00CF00E6A100E0D6E4EEC4EF000095B
:103DD80001E062D65ED0146A156A166A176A0A0E7E
:103DE80012EC51F0000955E141C00BF042C00CF053
:103DF8000E6A100E0D6E4EEC4EF0E9D7146A156A75
:103E0800166A176A3A0E12EC51F0000942E1040EE4
:103E1800406E0AD016EC53F041C0D9FF42C0DAFF19
:103E2800DF6E414A422A4006405001E135D6F2D7BA
:103E3800146A156A166A176A8D0E12EC51F0000999
:103E480028E116EC53F041C00BF042C00CF00E6AAA
:103E5800400E0D6E4EEC4EF0BAD7040E3F6E19D0E0
:103E68001A501D6E1E6A1E50F8E11D5001E10FD652
:103E7800010A01E113D6020A01E1C8D6090A8EE057
:103E8800010A93E0070AA7E0010AB8E0030AD0E0B4
:103E9800E4D72EEC53F03F50120055C058F056C0EE
:103EA80059F001017C6B7D6BF6D154C046F0580E79
:103EB800476E57C048F04750D96EDA6ADECFF6FF32
:103EC800DDCFF7FFF86A000EF86E0800F550250AF6
:103ED800D8A4C3D14750D96EDA6ADE2A000EDD2293
:103EE80001017E6B7F6B826B836B806981694750B0
:103EF800D96EDA6ADECFF6FFDDCFF7FFF86A000E7B
:103F0800F86E0800F550780AD8B40FD04750D96E2B
:103F1800DA6ADECFF6FFDDCFF7FFF86A000EF86E3B
:103F28000800F550580AD8A46ED14750D96EDA6AFD
:103F3800DECFF6FFDDCFF7FFF86A000EF86E080057
:103F4800F5CF53F04750D96EDA6ADE2A000EDD222B
:103F58004850D96EDA6ADF50DF2ADF2AD96EDA6A6A
:103F6800DECF49F0DDCF4AF049C04BF04AC04CF0F3
:103F78004D6A4E6A4F6A506A516A526A46C024F0C6
:103F88004BC025F04CC026F04DC027F04EC028F09D
:103F98004FC029F050C02AF051C02BF052C02CF06D
:103FA80053C02DF081BF01D0829381BF05D08151CC
:103FB80007E18005D8B004D0376A010E366E04D008
:103FC80080C136F081C137F07EC140F07FC141F039
:103FD80082A904D0FE0E4026FF0E412225C038F0EB
:103FE80026C039F027C03AF028C03BF029C03CF081
:103FF8002AC03DF02BC03EF02CC03FF0436A1F0E94
:10400800426E02019F6B6DD04206D8A043060F0E88
:104018003814446E456A45BE08D0455004E10A0E7E
:10402800445CD8A002D0570E01D0300E4426000EB2
:104038004522BF0E2E6E2F682D50306E316A2E50DD
:1040480030262F503122315005E11A0E305C02E241
:10405800010E01D0000E326E336A32503310D8B4DC
:1040680025D09F0E2E6E2F68200E4410306E000E45
:104078004510316E2E5030262F503122315005E137
:104088001A0E305C02E2010E01D0000E346E356A61
:1040980034503510D8B40AD044C011F045C012F0DD
:1040A800BDEC4FF011C044F012C045F0800E422420
:1040B800D96E020E4320DA6E44C0DFFF3606D8A060
:1040C80037064006D8A04106040E2E6ED8903F321F
:1040D8003E323D323C323B323A32393238322E2E81
:1040E800F5D743BE21D0435004E1020E425CD8A06C
:1040F8001BD0385039103A103B103C103D103E1080
:104108003F10D8A481D737BE05D0375002E1360416
:10411800D8B07AD741BE08D0415003E14004D8A0B6
:1041280003D0010182B370D7010182A916D04206DB
:10413800D8A04306800E4224D96E020E4320DA6EC0
:104148002DC0DFFF4206D8A04306800E4224D96E58
:10415800020E4320DA6E300EDF6E24C01AF0800E95
:1041680042241B6E020E43201C6E40C01DF041C04D
:104178001EF082A108D01BC014F01CC015F01AC094
:1041880016F093EC51F01EBE05D01DC022F01EC0E3
:1041980023F002D0226A236A206A216A0AD0000E1C
:1041A8000D6E200E0C6E1AC00EF0FDEC4AF0204A7F
:1041B800212A2250205C2150800A1F6E2350800A39
:1041C8001F58D8A0ECD7010182B108D01BC014F049
:1041D8001CC015F01AC016F093EC51F01BC00BF080
:1041E8001CC00CF021EC50F022500B241A6E235006
:1041F8000C201B6E1AC024F01BC025F024C046F00A
:1042080025C047F043D04750D96EDA6ADECFF6FFB3
:10421800DDCFF7FFF86A000EF86E0800F550250AA2
:10422800D8A412D04750D96EDA6ADE2A000EDD22F1
:10423800000E0D6E250E0C6E46C00EF0FDEC4AF019
:10424800476A010E466E22D04750D96EDA6ADE2AD6
:10425800000EDD22466A476A19D04750D96EDA6ADD
:10426800DECFF6FFDDCFF7FFF86A000EF86E080024
:10427800F5500C6E0D6A46C00EF0FDEC4AF0475042
:10428800D96EDA6ADE2A000EDD22DAD7465001013D
:104298007C2747507D2358C0F6FF59C0F7FF080018
:1042A800F55001E002D67CC154F07DC155F01200F2
:1042B80020EE04F0A351D926A451DA22DECFA7F0CC
:1042C800DDCFA8F0A729B06F000EA821B16FB011FB
:1042D800D8B4040C20EE0EF0A351D926A451DA224A
:1042E800DE50DE10DE10DE1001E1040CB0C0A7F0D5
:1042F8000F0EA71701E094D120EE0EF0A351D92696
:10430800A451DA22DE2A000EDE22DE22DE2220EE90
:104318000AF0A351D926A451DA22DE50DE10DE10AD
:10432800DE1011E1A3C0D9FFA4C0DAFF10EE08F037
:10433800DE50E126DD50E222E650B05DE650B1598C
:1043480001E26ED1040CB0C0A7F0B1C0A8F0040E11
:10435800A96FD890A833A733A92FFBD7AA69AB694F
:10436800A3C0D9FFA4C0DAFF10EE02F0DE50E126A8
:10437800DD50E222E750AC6FAD6BAA51AC27AB51D0
:10438800AD23A751AC17A851AD17AC51AD1101E041
:1043980047D1A3C0D9FFA4C0DAFFDECF44F0DDCFF8
:1043A80045F020EE0AF0A351D926A451DA22DECF37
:1043B80046F0DECF47F0DECF48F0DECF49F028ECFC
:1043C8001BF044C0B2F045C0B3F046C0B4F047C0DB
:1043D800B5F00001B551B411B31104E1020EB25D9C
:1043E80001E2020CB22907E1B32905E1B42903E18E
:1043F800B52901E1010CA3C0D9FFA4C0DAFF10EE72
:1044080012F0DE50E126DD50E222E650B25DE650C1
:10441800B359E650B459E650B55901E2D2D0A55186
:10442800A61101E1040CA3C0D9FFA4C0DAFFDECFB6
:104438008CF0DDCF8DF020EE0AF0A351D926A451DF
:10444800DA22DECF8EF0DECF8FF0DECF90F0DECF37
:1044580091F028EC2DF08CC0B2F08DC0B3F08EC076
:10446800B4F08FC0B5F0B251B311B411B51101E178
:10447800070CB205B311B411B51101E1020CB22950
:1044880007E1B32905E1B42903E1B52901E1010CEC
:10449800A3C0D9FFA4C0DAFFDECF24F0DDCF25F01A
:1044A80042EC3FF0000901E0010CA3C0D9FFA4C011
:1044B800DAFFDECFA7F0DDCFA8F02E0E0001A7258A
:1044C8000B6E000EA8210C6E0E6A0D6A020E106E9D
:1044D8000F6A2DEC52F0A3C0D9FFA4C0DAFFDECFDB
:1044E8000BF0DDCF0CF0B2C00DF0B3C00EF0B4C0CD
:1044F8000FF0B5C010F05FEC43F0A3C0D9FFA4C023
:10450800DAFF10EE2AF0DE50E126DD50E2220BC081
:10451800E6FF0CC0E6FF0DC0E6FF0EC0E6FF000197
:10452800AE6BAF6B2BD0A3C0D9FFA4C0DAFF10EEDF
:1045380004F0DE50E126DD50E222010EE76EA3C052
:10454800D9FFA4C0DAFFDECF24F0DDCF25F042EC9E
:104558003FF0000901E0010CA3C0D9FFA4C0DAFFB5
:1045680010EE2AF0DE50E126DD50E222E62A000EA7
:10457800E622E622E6220001AE4BAF2BA3C0D9FF0C
:10458800A4C0DAFF10EE02F0DE50E126DD50E22290
:10459800E750A76FA86BA751AE5DA851AF59C3E309
:1045A800A3C0D9FFA4C0DAFF10EE2AF0DE50E1263E
:1045B800DD50E222AE51E65EAF51E65A000EE65AF1
:1045C800E65A20EE0AF0A351D926A451DA22B2C045
:1045D800DEFFB3C0DEFFB4C0DEFFB5C0DEFFA3C0A0
:1045E800D9FFA4C0DAFFDECF0BF0DDCF0CF0B2C0EC
:1045F8000DF0B3C00EF0B4C00FF0B5C010F05FEC12
:1046080043F0000120EE0EF0A351D926A451DA227E
:104618000BC0DEFF0CC0DEFF0DC0DEFF0EC0DEFFEC
:1046280020EE04F0A351D926A451DA22B0C0DEFF4F
:10463800B1C0DDFF0F0EB015A76FA86B050ED8909F
:10464800A737A837E82EFBD7A3C0D9FFA4C0DAFF45
:10465800DECFA9F0DDCFAAF0A751A927A851AA2338
:104668002E0EA927000EAA2320EE12F0A351D92658
:10467800A451DA22A9C0DEFFAAC0DDFF000C18C0D1
:10468800F6FF19C0F7FF0800F5CF46F0184A192AB7
:10469800465001E11200250E461804E04650E7ECAA
:1046A80052F0EDD7416A426A18C0F6FF19C0F7FF09
:1046B8000800F5CF46F0184A192A300E46180DE1C1
:1046C800426A010E416E18C0F6FF19C0F7FF0800D4
:1046D800F5CF46F0184A192A06D02D0E461803E1E0
:1046E800426A020EEFD7396A3A6A1CD00A0E3902BA
:1046F800F3CF1BF0F4CF1CF03A02F3501C264650BF
:104708001B26000E1C22D00E1B24396EFF0E1C2007
:104718003A6E18C0F6FF19C0F7FF0800F5CF46F04B
:10472800184A192A2F0E466403D0390E4664DED77C
:104738006C0E461803E04C0E46180AE1418418C076
:10474800F6FF19C0F7FF0800F5CF46F0184A192AF6
:10475800465001E1120046C045F0600E456472D033
:10476800200E455E6FD01A50D96EDA6A020EDF2627
:10477800DF5CD96EDA6ADECF35F0DECF36F03B6A21
:104788003C6A02D03B4A3C2A3B5035241B6E3C50C5
:1047980036201C6E1BC0F6FF1CC0F7FF000EF86E1B
:1047A8000F0EF76403D00800F55005D0F6CFE9FFE7
:1047B800F7CFEAFFEF50000904E0E4D7200EE7EC5A
:1047C80052F041B20BD03B501B6E3C501C6E3B4A22
:1047D8003C2A39501B5C3A501C58F0E335C00CF0A9
:1047E80036C00DF0CEEC4EF003D0200EE7EC52F0C0
:1047F8003B501B6E3C501C6E3B4A3C2A39501B5C9C
:104808003A501C5801E33BD7F0D71A50D96EDA6AF0
:10481800DF50DF2ADF2AD96EDA6ADF50E7EC52F080
:104828002ED7386A020E08D0386A080E05D0386AC2
:104838000A0E02D0386A100E376E19D04650E7ECCF
:1048480052F01DD745501B6E1C6A1C50F7E11B50D7
:10485800420AE7E0010AD9E0070AE9E00B0AE4E0C6
:104868001C0A81E0060AE3E00D0AE4E0E7D741B458
:1048780030D0440E451813E01A50D96EDA6ADF506A
:10488800DF2ADF2AD96EDA6ADECF1BF0DDCF1CF013
:104898001BC02DF01CC02EF02F6A306A11D01A50A0
:1048A800D96EDA6ADF50DF2ADF2AD96EDA6ADECFFC
:1048B8002DF0DDCF2EF0000E2EBEFF0E2F6E306EC7
:1048C8002DC03DF02EC03EF02FC03FF030C040F06C
:1048D80010D01A50D96EDA6A040EDF26DF5CD96E62
:1048E800DA6ADECF3DF0DECF3EF0DECF3FF0DECF3E
:1048F80040F0440E45180CE140AE0AD03D6C3E1E17
:10490800D8B03E2A3F1ED8B03F2A000E40564186F6
:10491800436A446A3DC00BF03EC00CF03FC00DF046
:1049280040C00EF037C00FF038C010F0116A126A9C
:1049380007EC4DF00B50456E3DC00BF03EC00CF03F
:104948003FC00DF040C00EF037C00FF038C010F077
:10495800116A126AC1EC4BF00BC03DF00CC03EF07E
:104968000DC03FF00EC040F0090E45640BD0780E24
:10497800461803E0326A070E02D0326A270E316EFB
:104988003150452643501D0FD96EDA6A4550300F15
:10499800DF6E434A442A3D503E103F10401005E068
:1049A800445003E1100E435CB5E341A608D04350E0
:1049B8001D0FD96EDA6A2D0EDF6E434A442A43C0B2
:1049C8003BF044C03CF041B003D0346A200E02D022
:1049D800346A300E336E33C045F003D04550E7ECEF
:1049E80052F041B20BD03B501B6E3C501C6E3B4A00
:1049F8003C2A39501B5C3A501C58F0E34306D8A0B7
:104A0800440643501D0FD96EDA6ADF50E7EC52F0C6
:104A18004350441004E0F2D7200EE7EC52F03B502C
:104A28001B6E3C501C6E3B4A3C2A39501B5C3A506A
:104A38001C5801E324D6F0D7106E0C5002E0FCECB1
:104A48004BF00F6A0B5001E16ED1109E040E101846
:104A580003E0140E101807E101018E6B8F6B0C6ACE
:104A6800070E0B6E070C3F0E101807E1706A010164
:104A78008E6B8F6B0B6A0C6A12005F0E101807E1C1
:104A8800716A01018E6B8F6B0B6A0C6A12003F0E04
:104A9800106406D05F0E106003D0400E1018F0E1CD
:104AA800400E101809E1010E716E706A01018E6BDB
:104AB8008F6B0B6A0C6A1200200E101801E033D1BC
:104AC800010E706EF3D7600E101808E1715006E001
:104AD8006F50080ED8B4030E0F6E72D0600E101807
:104AE80008E1705006E06F5002E0090E14D0050E80
:104AF80012D0680E101809E1705007E01A0E010173
:104B08008F6F900E04D1898068D1680E101805E166
:104B1800715003E0020E0F6E53D06A0E101807E1B1
:104B2800705005E01A0E01018F6FF40EF0D06C0E74
:104B3800101807E1705005E01A0E01018F6F2C0E56
:104B4800E6D0700E101808E1715006E0040E0F6EE2
:104B580001018E6B8F6BD7D7700E101801E03DD115
:104B6800705001E13AD11B0E01018F6F620ECFD058
:104B78008980020E101805E11A0E01018F6F920E3E
:104B88008E6F050E101805E11A0E01018F6FAE0E1B
:104B98008E6F070E101805E11A0E01018F6FB80EFF
:104BA8008E6F080E101805E11A0E01018F6FCC0EDA
:104BB8008E6F030E101802E0102806E10F6A899024
:104BC80001018E6B8F6B09D1160E101801E005D10B
:104BD8001A0E01018F6FA40E8BD0050E101801E07C
:104BE800FCD01A0E01018F6FF50E82D010C073F041
:104BF8001A0E01018F6F9B0E7BD01A0E01018F6F69
:104C08009C0E76D07350070D500EF324D96E010E0A
:104C1800F420DA6E10C0DFFF1A0E01018F6F9D0EAF
:104C280067D07350070D510EF324D96E010EF4208E
:104C3800DA6E10C0DFFF1A0E01018F6F9E0E58D07A
:104C48007350070D520EF324D96E010EF420DA6E5C
:104C580010C0DFFF01018E6B8F6B010E17D01A0E8B
:104C680001018F6FB90E53D01A0E01018F6FBA0E62
:104C78003FD01A0E01018F6FBB0E3AD001018E6B27
:104C88008F6B3DD001018E6B8F6B060E0F6EA5D01A
:104C980010C073F001018E6B8F6B0F6A30D06F6A92
:104CA8001A0E01018F6FF70E8E6F29D01A0E0101AF
:104CB8008F6FF70E1DD08990270E01018F6F0F0E91
:104CC80017D0180E101801E088D01A0E01018F6F46
:104CD8002D0E0ED01A0E01018F6F2E0E09D01A0E4E
:104CE80001018F6F2F0E04D01A0E01018F6F300E45
:104CF8008E6F73D001018E6B8F6B0A0E0F6E8990C9
:104D08006CD0040E0F6E270E01018F6F0F0E8E6F81
:104D1800FAD6898003D08990010E6F6E01018E6BDF
:104D28008F6B0F6A5AD08EC10DF08FC10EF00E50E6
:104D380007E01A0A09E0010A48E03C0A4CE04DD0B5
:104D48000D5001E1C0D649D00D502C0ABAE0010A35
:104D5800C1E0030AC4E0010AC7E01F0ACBE0A00AC9
:104D680001E106D7020A01E141D7090A01E145D765
:104D7800070A01E147D7010A01E153D7030A01E114
:104D88005FD73A0A01E17ED70A0AC5E0160A01E1AF
:104D980066D7010A01E168D7030A01E16AD7010A67
:104DA80001E16CD7790A01E1B5D60E0A01E170D7A5
:104DB800380A01E112D7010A01E171D7030A01E1BA
:104DC80075D7010A01E177D708D00D50580A99E044
:104DD8003A0A9FE002D00D500F0A0FC00BF00C6A80
:104DE8001200000E626E020E636E340E646E0A0EBE
:104DF800656E020E676E666ADD0E686E696A4DEC56
:104E080011F06C6EE70E0001806FFD0E816FDDC042
:104E180082F0DEC083F0DDEC52F00001DF6BE06B66
:104E2800DB6BDC6BE16BE26BE151BD0FD96EDA6ACB
:104E3800DF6AE151CC0FD96EDA6A000EDF6EE14B02
:104E4800E22BE2BFF1D7E25103E10F0EE15DECE3A3
:104E5800E36BE46B1CD1340EE325D96E0A0EE42112
:104E6800DA6E0D0EDE1801E0D7D08F0E0B6EFF0E36
:104E78000C6EBD0E0D6E97EC49F00B500C1007E14F
:104E8800CC0E126E68EC44F012500101FC6F890ED2
:104E98000B6EFF0E0C6EBD0E0D6E97EC49F00B50AD
:104EA8000C1007E1CC0E126E68EC44F012500101B0
:104EB800A06F670E0B6EFF0E0C6EBD0E0D6E97EC9D
:104EC80049F00B500C1007E1CC0E126E68EC44F060
:104ED80012500101986FD40E0B6EFF0E0C6EBD0EB2
:104EE8000D6E97EC49F00B500C1007E1CC0E126ECA
:104EF80068EC44F012500101966F0001E56BE66B17
:104F0800AE0E5A6E5B6A6E0E5C6EFF0E5D6EE5C08D
:104F18005EF0E6C05FF0F6EC50F0AE0E0B6E0C6A79
:104F2800BD0E0D6E97EC49F00B500C1017E10F0EEB
:104F38000001E503F3CFACF0F4CFADF0E603F35096
:104F4800AD27340EAC250B6E0C0EAD210C6ECC0EBD
:104F58000D6E0F6A0F0E0E6E4AEC4FF00001E54B16
:104F6800E62BE6BFCDD7E65103E1100EE55DC8E3B9
:104F7800E66B010EE56FAE0E5A6E5B6A750E5C6EDF
:104F8800FF0E5D6EE5C05EF0E6C05FF0F6EC50F037
:104F9800AE0E0B6E0C6ABD0E0D6E97EC49F00B5001
:104FA8000C1017E10F0E0001E503F3CFACF0F4CFBE
:104FB800ADF0E603F350AD27240EAC250B6E0D0EB5
:104FC800AD210C6ECC0E0D6E0F6A0F0E0E6E4AECF4
:104FD8004FF00001E54BE62BE6BFCDD7E65103E1E4
:104FE800040EE55DC8E3E16BE26BE151BD0FD96EDC
:104FF800DA6ADF6AE151CC0FD96EDA6A000EDF6E29
:10500800E14BE22BE2BFF1D7E25103E10F0EE15D84
:10501800ECE3DB6BDC6B15D0340EE325D96E0A0E9E
:10502800E421DA6E0A0EDE1830E0340EE325D96E7C
:105038000A0EE421DA6E200EDE1806E1DC6B010EA2
:10504800DB6FDF6BE06B21D0DB51DC1109E0340E44
:10505800E325D96E0A0EE421DA6EDF51CC0F08D0B1
:10506800340EE325D96E0A0EE421DA6EDF51BD0F46
:10507800E16EE26ADFCFE7FFE0BF05D0E05105E16E
:105088000F0EDF5D02E2DF4BE02BE34BE42BDD513B
:10509800E35DDE51E45901E2DED6D70E806FFD0EE6
:1050A800816F98C182F0836BDDEC52F0350E000100
:1050B800806FFE0E816FFCC182F0836BDDEC52F0D5
:1050C800260E0001806FFE0E816FA0C182F0836BF7
:1050D800DDEC52F00001E56BE66B630E806FFD0EB0
:1050E800816FE5C082F0E6C083F00F0EE503F3CFD1
:1050F800ACF0F4CFADF0E603F350AD27340EAC2599
:10510800846F0C0EAD21856FDDEC52F00001E54B8C
:10511800E62BE6BFE2D7E65103E1100EE55DDDE3DD
:10512800E46B010EE36F740E806FFD0E816FE3C0B8
:1051380082F0E4C083F00F0EE303F3CFACF0F4CFBA
:10514800ADF0E403F350AD27240EAC25846F0D0EAB
:10515800AD21856FDDEC52F00001E34BE42BE4BF99
:10516800E2D7E45103E1040EE35DDDE3730E806FE3
:10517800FB0E816FDDEF52F043C024F044C025F0F0
:1051880042EC3FF04D6E4D5001E08ED143C0D9FF47
:1051980044C0DAFF030EDE1801E076D120EE05F0F8
:1051A8004350D9264450DA22DE0401E06DD12E0E98
:1051B80043240B6E000E44200C6E0E6A0D6A020E1C
:1051C800106E0F6A2DEC52F022EE2CF04350D926C7
:1051D8004450DA22550EDF6E22EE2DF04350D926C8
:1051E8004450DA22AA0EDF6E20EE2EF04350D92664
:1051F8004450DA22520EDF6E20EE2FF04350D926AB
:105208004450DA22520EDF6E20EE30F04350D92699
:105218004450DA22610EDF6E20EE31F04350D92679
:105228004450DA22410EDF6E22EE12F04350D926A6
:105238004450DA22720EDF6E22EE13F04350D92664
:105248004450DA22720EDF6E22EE14F04350D92653
:105258004450DA22410EDF6E22EE15F04350D92673
:105268004450DA22610EDF6E20EE0EF04350D9264C
:105278004450DA2212EE16F04350E1264450E2225E
:10528800DFCFE7FF22EE17F04350D9264450DA2249
:1052980010EE0EF04350E1264450E222E6CF45F0EE
:1052A800E5CF46F046C045F0466A4550DF6E22EE2F
:1052B80018F04350D9264450DA2210EE0EF043502D
:1052C800E1264450E222E6CF45F0E6CF46F0E6CFAD
:1052D80047F0E6CF48F0110E05D0D8904832473253
:1052E80046324532E82EF9D74550DF6E22EE19F0E6
:1052F8004350D9264450DA2210EE0EF04350E126EE
:105308004450E222E6CF45F0E6CF46F0E6CF47F03C
:10531800E6CF48F0190E05D0D890483247324632C9
:105328004532E82EF9D74550DF6E20EE0AF043509B
:10533800D9264450DA2212EE1AF04350E12644509E
:10534800E222DFCFE7FF22EE1BF04350D92644507C
:10535800DA2210EE0AF04350E1264450E222E6CF6A
:1053680045F0E5CF46F046C045F0466A4550DF6E49
:1053780022EE1CF04350D9264450DA2210EE0AF0EF
:105388004350E1264450E222E6CF45F0E6CF46F00E
:10539800E6CF47F0E6CF48F0110E05D0D890483256
:1053A800473246324532E82EF9D74550DF6E22EEB5
:1053B8001DF04350D9264450DA2210EE0AF043502B
:1053C800E1264450E222E6CF45F0E6CF46F0E6CFAC
:1053D80047F0E6CF48F0190E05D0D890483247324A
:1053E80046324532E82EF9D74550DF6E20EE1AF0E6
:1053F8004350D9264450DA22DECF45F0DECF46F0BE
:10540800DECF47F0DECF48F04528496E000E462033
:105418004A6E000E47204B6E000E48204C6E20EE60
:105428002AF04350D9264450DA2249C0DEFF4AC048
:10543800DEFF4BC0DEFF4CC0DEFF2E0E43241A6E8B
:10544800000E44201B6E20EE2AF04350D92644500B
:10545800DA22DECF1CF0DECF1DF0DECF1EF0DECF6D
:105468001FF0216A010E206E20EE01F04350D9266C
:105478004450DA22DF50DBEC45F020EE05F04350D3
:10548800D9264450DA22DF6A1A6A1B6A1C6A20EE9F
:1054980001F04350D9264450DA22DF503EEC1DF08B
:1054A800000902E0010E4D6E4D5012008980B3ECE8
:1054B8003BF0CAC0A8F1CBC0A9F10101A851A911BC
:1054C8001AE07350140D130EF324D96E010EF42054
:1054D800DA6E7350140D130EF324E16E010EF420EE
:1054E800E26EE7500409DF6EC0EC51F0A8C1E1F0AC
:1054F800A9C1E2F012007350140D070EF324D96EFF
:10550800010EF420DA6E78C1E8F079C1E9F07AC1C9
:10551800EAF00001E76B000EE725EB6F010EE821CA
:10552800EC6F000EE921ED6F000EEA21EE6FDE5000
:10553800EB193BE1DE50EC1938E1DE50ED1935E1AD
:10554800DE50EE1932E16FEC4CF00FC0ACF110C038
:10555800ADF111C0AEF112C0AFF1000EE8CF34FAD0
:105568002AEE35F0AFC1DFFFE8CF36FA2AEE37F082
:10557800AEC1DFFFE8CF38FA2AEE39F0ADC1DFFF60
:10558800E8CF3AFA2AEE3BF0ACC1DFFF0101FA930B
:10559800010E496E486A56EC35F0FA936B6A8990A9
:1055A8006BC0E1F00001E26B12007350140D0F0E96
:1055B800F324D96E010EF420DA6EDECFE3F0DECFED
:1055C800E4F0DECFE5F0DECFE6F0E4C0E3F0E5C0DE
:1055D800E4F0E6C0E5F0E66BE3C0A1F1E4C0A2F1B7
:1055E8007350140D0F0EF324D96E010EF420DA6EE9
:1055F800DECFE3F0DDCFE4F0E3510101AA6FAB6B3E
:10560800FA93A66BA76BA36BA46B65D0E369E469F7
:10561800A1C1E5F0A2C1E6F0E351E527E451E62394
:105628000101A3510001E5190AE10101A45100019A
:10563800E61905E10101AA51AB1101E1FA837350A2
:10564800200D000EF324626E020EF420636E340EF9
:10565800646E0A0E656E010E676E666AB00E686E3D
:10566800010E696E4DEC11F00101A56FA55101E025
:1056780028D7B0C148F0B1C149F056EC35F0B05167
:10568800A627B151A7237350140D070EF324D96E22
:10569800010EF420DA6E000EDE240001E36F010E25
:1056A800DE20E46F000EDE20E56F000EDE20E66FE0
:1056B8007350140D070EF324D96E010EF420DA6E20
:1056C800E3C0DEFFE4C0DEFFE5C0DEFFE6C0DEFFCC
:1056D8000101A34BA42BA151A35DA451800A000191
:1056E800E36F0101A251800A0001E3598FE3010130
:1056F800ABBF4FD0AB5102E1AA054BE37350200D6D
:10570800000EF324626E020EF420636E340E646E93
:105718000A0E656EAAC166F0ABC167F0B00E686E7E
:10572800010E696E4DEC11F00101A56FA55101E064
:10573800C8D6FA83AAC148F0ABC149F056EC35F097
:10574800B051A627B151A7237350140D070EF324A7
:10575800D96E010EF420DA6E000EDE240001E36F2C
:10576800010EDE20E46F000EDE20E56F000EDE2065
:10577800E66F7350140D070EF324D96E010EF42052
:10578800DA6EE3C0DEFFE4C0DEFFE5C0DEFFE6C0A0
:10579800DEFF010102D71550D96EDA6ADECF22F09A
:1057A800DDCF23F002D0224A232A22C0F6FF23C0ED
:1057B800F7FF000EF86E0F0EF76403D00800F550DF
:1057C80005D0F6CFE9FFF7CFEAFFEF502F0AEBE05D
:1057D80022C0F6FF23C0F7FF000EF86E0F0EF76425
:1057E80003D00800F55005D0F6CFE9FFF7CFEAFF60
:1057F800EF505C0AD8E020EE14F01350D92614506C
:10580800DA22DECF24F0DDCF25F024C00BF025C04E
:105818000CF00E6A200E0D6E106A0B0E0F6E2DEC3A
:1058280052F01E6A1EC026F0276A26C01CF027C048
:105838001DF0206A080E1F6E1C502224166E1D5083
:105848002320176E16C0F6FF17C0F7FF000EF86E7C
:105858000F0EF76403D00800F55005D0F6CFE9FF26
:10586800F7CFEAFFEF50286E1C4A1D2A200E286445
:10587800A7D02F0E281801E1A3D05C0E281801E14B
:105888009FD02E0E281805E01F50265C2050275860
:1058980014E3080E1F182010D8A4060C2E0E281882
:1058A80001E0060C276A080E266E206A0B0E1F6E92
:1058B800D8901E36D8901E36BFD77F0E286402D0E7
:1058C800030E1E12800E286403D09F0E286406D093
:1058D800DF0E28644CD0FD0E286049D01C502224CD
:1058E800166E1D502320176E16C0F6FF17C0F7FF5F
:1058F800000EF86E0F0EF76403D00800F55005D0BF
:10590800F6CFE9FFF7CFEAFFEF50216E1C4A1D2AB8
:105918003F0E216403D07E0E216406D07F0E2164E1
:10592800060CFD0E2160060C166817681FC018F0DB
:1059380020C019F016501826175019221850265C46
:105948001950275801E3060C26502424D96E2750F5
:105958002520DA6E28C0DFFF264A272A265024246D
:10596800D96E27502520DA6E21C0DFFF26D0800EA1
:105978000B6EFE0E0C6E28C00DF00E6ADAEC50F0BD
:105988000B500C1001E0060C400E286405D05B0E8D
:10599800286002D01E8209D0600E286406D07B0ED3
:1059A800286003D01E80200E285E26502424D96E3D
:1059B80027502520DA6E28C0DFFF264A272A3CD741
:1059C8001C502224166E1D502320176E1550D96EB8
:1059D800DA6A16C0DEFF17C0DDFF200E286403D088
:1059E8001A6A1B6A03D01B6A040E1A6E1AC028F0C2
:1059F8002650271001E1060C24C0D9FF25C0DAFF84
:105A0800E50EDE1806E124C0D9FF25C0DAFF050E31
:105A1800DF6E080E1F18201004E1D8901E36D890AB
:105A28001E361E50030BE80601E128881E500C0B99
:105A3800040A01E1288620EE0BF02450D9262550CF
:105A4800DA2228C0DFFF000C8E518F1190119111BE
:105A580028E120EE0AF08C51D9268D51DA22DECFCA
:105A680097F0DECF98F0DECF99F0DECF9AF097511D
:105A7800981199119A110FE020EE12F08C51D92645
:105A88008D51DA22DE50975DDE509859DE509959D3
:105A9800DE509A5952E3010E976F986B996B9A6B87
:105AA8004CD08CC044F08DC045F08EC046F08FC0FD
:105AB80047F090C048F091C049F028EC1BF044C072
:105AC8009FF045C0A0F046C0A1F047C0A2F0000179
:105AD800A251A111A01109E1020E9F5D06E2010E7B
:105AE8008C6F8D6B8E6B8F6B000C9F290FE1A0293B
:105AF8000DE1A1290BE1A22909E19FC08CF0A0C00A
:105B08008DF0A1C08EF0A2C08FF0120020EE12F02E
:105B18008C51D9268D51DA22DE509F5DDE50A05976
:105B2800DE50A159DE50A259E8E38EC097F08FC02D
:105B380098F090C099F091C09AF097C09BF098C0E7
:105B48009CF099C09DF09AC09EF09B2B000E9C2360
:105B58009D239E2320EE12F08C51D9268D51DA22F6
:105B6800DE509B5DDE509C59DE509D59DE509E599B
:105B780011E3020E9B6F9C6B9D6B9E6B9A51991162
:105B8800981108E1020E975D05E28C6B8D6B8E6BA8
:105B98008F6B12008CC044F08DC045F09BC046F05E
:105BA8009CC047F09DC048F09EC049F028EC1BF00F
:105BB80044C09FF045C0A0F046C0A1F047C0A2F085
:105BC80000019F51A011A111A2111AE09F2906E11D
:105BD800A02904E1A12902E1A2298FE09F05A011D3
:105BE800A111A2118AE097519B19AFE198519C1914
:105BF800ACE199519D19A9E19A519E19C6E0A5D722
:105C08008CC044F08DC045F09BC046F09CC047F066
:105C18009DC048F09EC049F04A684B684C680F0E1A
:105C28004D6ECBEC18F0966F96511CE18E518F118A
:105C38009011911117E08CC044F08DC045F08EC0D2
:105C480046F08FC047F090C048F091C049F09BC023
:105C58004AF09CC04BF09DC04CF09EC04DF0CBEC80
:105C680018F0966F965130E120EE0AF08C51D92643
:105C78008D51DA229BC0DEFF9CC0DEFF9DC0DEFF97
:105C88009EC0DEFF20EE0EF08C51D9268D51DA220F
:105C9800DE2806E1DE2804E1DE2802E1DE2821E034
:105CA80020EE0EF08C51D9268D51DA22DE06000E38
:105CB800DE5ADE5ADE5A20EE05F08C51D9268D5177
:105CC800DA22000EDB800DD0960507E0010E9B6FEF
:105CD800000E9C6B9D6B9E6B04D09B699C699D69B3
:105CE8009E699BC08CF09CC08DF09DC08EF09EC0BC
:105CF8008FF0120020EE04F06250D9266350DA22A9
:105D080064C0DEFF65C0DDFF20EE06F06250D926D4
:105D18006350DA22DECF99F0DECF9AF0DECF9BF027
:105D2800DECF9CF0000199059A119B119C11D8B403
:105D3800020C62C0D9FF63C0DAFF10EE12F0DE5029
:105D4800E126DD50E222E650995DE6509A59E65088
:105D58009B59E6509C5901E3020C99519A119B11E9
:105D68009C1121E162C0D9FF63C0DAFFDECF8CF05D
:105D7800DDCF8DF08CC0D9FF8DC0DAFF030EDE18A1
:105D880012E162C0D9FF63C0DAFF10EE22F0DE50E4
:105D9800E126DD50E222E6CF99F0E6CF9AF0E6CF91
:105DA8009BF0E6CF9CF099519A119B119C1123E12D
:105DB80062C0D9FF63C0DAFF10EE08F0DE50E126BA
:105DC800DD50E222E650645CE650655801E3020CBF
:105DD80062C0D9FF63C0DAFF10EE22F0DE50E12680
:105DE800DD50E222E6CF95F0E6CF96F0E6CF97F0C9
:105DF800E6CF98F074D062C0D9FF63C0DAFF10EE26
:105E080002F0DE50E126DD50E222E750100DF3CF1C
:105E180093F0F4CF94F044D062C0D9FF63C0DAFFA6
:105E2800DECF44F0DDCF45F099C046F09AC047F088
:105E38009BC048F09CC049F028EC1BF044C099F086
:105E480045C09AF046C09BF047C09CF000019929D4
:105E580007E19A2905E19B2903E19C2901E1010C4D
:105E68009C519B119A1104E1020E995DD8A0020C75
:105E780062C0D9FF63C0DAFF10EE12F0DE50E126EF
:105E8800DD50E222E650995DE6509A59E6509B595A
:105E9800E6509C5901E3020C9351645E9451655A93
:105EA8009351645C94516558B7E262C0D9FF63C0EE
:105EB800DAFFDECF0BF0DDCF0CF099C00DF09AC001
:105EC8000EF09BC00FF09CC010F05FEC43F00BC0CD
:105ED80095F00CC096F00DC097F00EC098F020EE2B
:105EE8000AF06250D9266350DA2299C0DEFF9AC0C0
:105EF800DEFF9BC0DEFF9CC0DEFF000195519611BE
:105F08009711981101E1020C64C08CF065C08DF006
:105F1800040E8E6FD8908D338C338E2FFBD78C5117
:105F280095258F6F8D519621906F000E9721916F57
:105F3800000E9821926F20EE0EF06250D926635021
:105F4800DA228FC0DEFF90C0DEFF91C0DEFF92C074
:105F5800DEFF0F0E64148C6F8D6B050ED8908C3796
:105F68008D37E82EFBD762C0D9FF63C0DAFFDECFDA
:105F78008EF0DDCF8FF08C518E278D518F232E0E12
:105F88008E27000E8F2320EE12F06250D926635020
:105F9800DA228EC0DEFF8FC0DDFF000C000E00018C
:105FA800F66F0A0EF56F000EF46F050EF36F28D129
:105FB800F66B140EF56F1CD1060E0C6EFD0E0D6EF1
:105FC800CEEC4EF082B204D00001F66B1E0EF56FD7
:105FD800150E0001F26F4B0EF16FBE0EE82EFED7C4
:105FE800F12FFCD7F22FFAD700F002D1E00E0C6E99
:105FF800FE0E0D6ECEEC4EF0060E0001D26F080EAE
:10600800D36F750ED46FFB0ED56FD66B4CEC49F081
:106018006C6E6C5021EC4FF06C50DAE10001F66BBD
:10602800230ED5D7440E0C6EFE0E0D6ECEEC4EF040
:10603800000E0001D26F020ED36F0F0ED46FFF0E49
:10604800D56F010ED66F68EC16F06C6E6C5021ECB3
:106058004FF06C5009E1F5EC26F0000E5B6E020E75
:106068005C6E49EC51F06C6E6C5021EC4FF0000EF8
:106078000001F66F280EF56F010198510CE1FB6BDA
:10608800340E5A6E0C0E5B6EC60E5C6EFE0E5D6EA6
:10609800F6EC50F00DD0FB0E0001806FFB0E816F07
:1060A80098C182F0836BFBC184F0856BDDEC52F004
:1060B800530E0001806FFE0E816F0101FB510F0D21
:1060C800340EF3240001826F0C0EF420836FDDEC94
:1060D80052F07ED7960E806FFC0E816F0101FB5146
:1060E8000F0D340EF3240001826F0C0EF420836F21
:1060F800DDEC52F0000E0001D26F020ED36F0101E9
:10610800FB510F0D340EF3240001D46F0C0EF42054
:10611800D56F030ED66F68EC16F06C6E6C5004E108
:106128000001F66B3C0EF56F040E6C1801E050D7B9
:106138000001F66B320E4BD7400E806FFD0E816F5B
:106148000101FB510F0D340EF3240001826F0C0E78
:10615800F420836FDDEC52F0000E0001D26F020EC6
:10616800D36F0101FB510F0D340EF3240001D46FDE
:106178000C0EF420D56F070ED66F68EC16F06C6E17
:106188006C5001E025D70001F66B3C0E20D71A0EA3
:10619800806FFD0E816F0101FB510F0D340EF3244A
:1061A8000001826F0C0EF420836FDDEC52F00001C9
:1061B800F06B010EEF6F010CF5C0F1F0F6C0F2F0D4
:1061C800F25116E1F1510A0A01E1F2D61E0A01E183
:1061D800F3D60A0A01E10AD73D0A01E123D70B0ADF
:1061E80001E178D7050A04E01F0AA6E00E0ACFE00D
:1061F800140E0001F519F61103E0F307D8A0F4070F
:10620800F4BF04D0F451D8E1F305D6E2EF6BF06B9C
:106218001200340E0101AD6F0A0EAE6FEAC00BF02A
:10622800EBC00CF021EC50F00B500101A16FCA0E2D
:106238000001A36FA46BA56BA66BA76BA86B63EC9F
:106248000EF00101AA6FAA510DE04D0E0001806FFA
:10625800FC0E816FDDEC52F00001CA6BCB6BCC6B8E
:10626800CD6B1200CA0E626E636AADC164F0AEC136
:1062780065F0010E676E666AA80E686E010E696E9B
:106288004DEC11F00101AA6FAA5108E0DB0E0001E4
:10629800806FFC0E816FDDEC52F0DED7ADC1D9FF07
:1062A800AEC1DAFF800EDE1808E0850E0001806FAF
:1062B800FD0E816FDDEC52F0CFD720EE0AF0AD5124
:1062C800D926AE51DA22DF500001ED6FEC6B0101E7
:1062D80020EE0BF0AD51D926AE51DA22DF50000185
:1062E800EC250101A66F000E0001ED210101A76F49
:1062F800C40E0001806FFC0E816FA6C182F0A7C199
:1063080083F0DDEC52F0CA0E0001A36FA46B01010B
:10631800A6510001ED6FEC6BECC0A5F0EDC0A6F046
:10632800A76BA86B63EC0EF00101AA6FAA5194E168
:10633800CA0E626E636AADC164F0AEC165F0010E4B
:10634800676E666AA80E686E010E696E4DEC11F0F4
:106358000101AA6FAA5180E1AB6BAC6BEAC00BF0EC
:10636800EBC00CF0ABC1ECF0ACC1EDF0050ED89071
:106378000001EC37ED37E82EFAD7EC510101AD25D5
:106388000D6E0001ED510101AE210E6EA1C10FF09D
:10639800106A2AEC4AF00B500C105DE1ABC1ECF02E
:1063A800ACC1EDF0050ED8900001EC37ED37E82EC2
:1063B800FAD7ADC1EEF0AEC1EFF0EC51EE27ED51DA
:1063C800EF230E0EEE25D96E000EEF21DA6EDF50A8
:1063D800F16FF06BABC1F2F0ACC1F3F0050ED890E1
:1063E800F237F337E82EFBD7ADC1F4F0AEC1F5F0C4
:1063F800F251F427F351F5230F0EF425D96E000E50
:10640800F521DA6EDF50F66FF76BF051F627F15190
:10641800F723F6C0A2F1F7C0A3F10101000EA3BF54
:10642800FF0EA46FA56F620E0001806FFE0E816FD4
:10643800A2C182F0A3C183F0A4C184F0A5C185F0F4
:10644800DDEC52F0A2C1CAF0A3C1CBF0A4C1CCF0DC
:10645800A5C1CDF01200AB4BAC2BACBF7FD7AC5174
:1064680005E10F0EAB5D01E3F7D678D7F5D6D30E6D
:106478000001806FFE0E816F4CC082F04DC083F02A
:1064880048C084F049C085F04AC086F04BC087F008
:10649800DDEC52F0546A556ACED0730E0001806F5D
:1064A800FB0E816FDDEC52F0566A576A29D054C052
:1064B8004EF055C04FF04E3A4F3AF00E4F164E5030
:1064C8000F0B4F12F00E4E1648C050F049C051F055
:1064D8004E5050264F50512256505024D96E575086
:1064E8005120DA6EDF50536E9B0E0001806FFF0E55
:1064F800816F53C082F0836BDDEC52F0564A572A05
:1065080057BE05D057501DE1100E565C1AE254C014
:106518004EF055C04FF04E3A4F3AF00E4F164E50CF
:106528000F0B4F12F00E4E1656504E2657504F2254
:106538004E504A5C4B50800A506E4F50800A50585B
:10654800B6E2E00E0001806FFF0E816FDDEC52F0C5
:10655800566A576A4DD054C04EF055C04FF04E3A67
:106568004F3AF00E4F164E500F0B4F12F00E4E16BC
:1065780048C050F049C051F04E5050264F5051225B
:1065880056505024D96E57505120DA6E200EDF64D1
:1065980026D0FC0E0001806FFF0E816F54C04EF0B4
:1065A80055C04FF04E3A4F3AF00E4F164E500F0B63
:1065B8004F12F00E4E1648C050F049C051F04E50E0
:1065C80050264F50512256505024D96E57505120C2
:1065D800DA6EDF50826F836BDDEC52F007D00D0E60
:1065E8000001806FFF0E816FDDEC52F0564A572A8A
:1065F80057BE05D057501DE1100E565C1AE254C024
:106608004EF055C04FF04E3A4F3AF00E4F164E50DE
:106618000F0B4F12F00E4E1656504E2657504F2263
:106628004E504A5C4B50800A506E4F50800A50586A
:1066380092E2544A552A55BE05D055501AE1500EDB
:10664800545C17E254C04EF055C04FF04E3A4F3AE2
:10665800F00E4F164E500F0B4F12F00E4E164A50BA
:106668004E5C4F50800A506E4B50800A505801E2E1
:1066780014D7730E0001806FFB0E816FDDEF52F0AF
:1066880020EE04F04450D9264550DA22DF6A20EE85
:106698002AF04450D9264550DA22DE68DE68DE68E2
:1066A800DD6844C039F045C03AF046C03BF047C009
:1066B8003CF048C03DF049C03EF0FEEC48F000090F
:1066C80001E0030C22EE2DF04450D9264550DA2281
:1066D800DF504B6E4A6A22EE2CF04450D9264550C2
:1066E800DA22DF504A12550E4A1803E1AA0E4B1857
:1066F80001E0020C20EE65F04450D9264550DA221C
:10670800DF504B6E4A6A20EE66F04450D926455059
:10671800DA22DF504C6E4CC04DF04E6A4F6A506A18
:106728004EC050F04DC04FF04E6A4D6A20EE67F0F3
:106738004450D9264550DA22DF50516E51C052F0EC
:10674800536A546A556A52C055F0546A536A526A79
:106758004D505210566E4E505310576E4F505410A5
:10676800586E50505510596E4A5056105A6E4B502C
:1067780057105B6E000E58105C6E000E59105D6E5F
:1067880020EE64F04450D9264550DA22DF505A10E2
:106798005E6E5B505F6E5C50606E5D50616E5E5009
:1067A800626E5F50636E6050646E656A460E621872
:1067B80008E1410E631805E1540E6418651001E103
:1067C800000C20EE81F04450D9264550DA22DF50E3
:1067D8004B6E4A6A20EE82F04450D9264550DA22A0
:1067E800DF504C6E4CC04DF04E6A4F6A506A4EC036
:1067F80050F04DC04FF04E6A4D6A20EE83F0445081
:10680800D9264550DA22DF50516E51C052F0536AF2
:10681800546A556A52C055F0546A536A526A4D50C8
:106828005210566E4E505310576E4F505410586EAB
:1068380050505510596E4A5056105A6E4B505710BA
:106848005B6E000E58105C6E000E59105D6E20EEE7
:1068580080F04450D9264550DA22DF505A105E6E37
:106868005B505F6E5C50606E5D50616E5E50626E34
:106878005F50636E6050646E656A460E621808E188
:10688800410E631805E1540E6418651001E1000C0F
:10689800010C4EC00CF04FC00DF071EC4AF0546E74
:1068A800545001E0FDD020EE04F04E50D9264F5050
:1068B800DA22DFAAF5D04EC0D9FF4FC0DAFFDECF0B
:1068C80039F0DDCF3AF020EE1AF04E50D9264F506D
:1068D800DA22DECF3BF0DECF3CF0DECF3DF0DECF7C
:1068E8003EF0FEEC48F0546E545001E0D9D020EE52
:1068F8001EF04E50D9264F50DA22DECF59F0DDCFA8
:106908005AF020EE0BF05950D9265A50DA22000ED0
:10691800DB8A20EE0AF04E50D9264F50DA2210EECC
:106928001CF05950E1265A50E222DFCFE7FF20EE53
:106938001DF05950D9265A50DA2210EE0AF04E505E
:10694800E1264F50E222E6CF50F0E5CF51F051C09A
:1069580050F0516A5050DF6E20EE1EF05950D92683
:106968005A50DA2210EE0AF04E50E1264F50E22239
:10697800E6CF50F0E6CF51F0E6CF52F0E6CF53F035
:10698800110E05D0D8905332523251325032E82E7F
:10699800F9D75050DF6E20EE1FF05950D9265A50C3
:1069A800DA2210EE0AF04E50E1264F50E222E6CFEE
:1069B80050F0E6CF51F0E6CF52F0E6CF53F0190E83
:1069C80005D0D8905332523251325032E82EF9D78E
:1069D8005050DF6E59C00BF05AC00CF020EE0EF08C
:1069E8004E50D9264F50DA22DECF0DF0DECF0EF012
:1069F800DECF0FF0DECF10F000EC50F0556A566A8B
:106A0800210E576E460E586E20EE16F05950D926B4
:106A18005A50DA22DF6A20EE17F05950D9265A5018
:106A2800DA2256C0DFFF20EE18F05950D9265A5006
:106A3800DA2257C0DFFF20EE19F05950D9265A50F4
:106A4800DA2258C0DFFF20EE12F05950D9265A50EA
:106A5800DA22DF6A20EE13F05950D9265A50DA228A
:106A6800DF6A20EE04F04E50D9264F50DA22DF0EAE
:106A7800DF164EC0D9FF4FC0DAFF10EE04F0DE502B
:106A8800E126DD50E222010EE76E4EC0D9FF4FC06D
:106A9800DAFFDECF43F0DDCF44F0C0EC28F0546ECF
:106AA8005450120001019D6B866B876B938693800F
:106AB80093829384938895688A908A928A948A9814
:106AC800010E9C6F898E89B40ED0E7A707D0760E89
:106AD8000001806FFB0E816FDDEC52F001019C6BB1
:106AE800486A496A1200F2981A0EE82EFED700D0BA
:106AF800BCD081B809D095689380710E0001806F71
:106B0800FE0E816FDDEC52F081B80BD0710E0001E2
:106B1800806FFE0E816FDDEC52F0630E01019D6FF8
:106B2800AAD0100E0101746F270E756F766B776B04
:106B380086D081B281A410D07407000E755B765B95
:106B4800775B742906E1752904E1762902E1772942
:106B5800D8A48BD0620E69D0010E67D081A885D0E9
:106B6800020E63D04A684B6848C04CF049C04DF0EB
:106B78004A504C264B504D2286514C1805E18751FE
:106B88004D1802E1FAB3939A340E8625D96E0A0E8F
:106B98008721DA6EDF1C8C6E864B872B956A030E75
:106BA8001ED0100E746F270E756F766B776B5DD0E5
:106BB80081B20DD07407000E755B765B775B742924
:106BC80008E1752906E1762904E1772902E1040E36
:106BD8009D6F81A24AD0040E28D09390050E9D6F18
:106BE800E0D7938481B40DD07407000E755B765B93
:106BF800775B742908E1752906E1762904E177298C
:106C080002E1060E9D6F81A430D0060E0ED0938A45
:106C1800938095684850865D8751800A4A6E49502E
:106C2800800A4A5899E3630E01019D6F1ED0A10E98
:106C38000001806FFF0E816FDDEC52F0F4D79D519B
:106C48004A6E4B6A4B5011E14A5001E172D7010A72
:106C580085E0030A87E0010AABE0070ABEE0010A03
:106C6800C0E0030AD4E0640AE2E0630E01019D1962
:106C780002E081BC3ED7F292F2889C6B93809382AB
:106C880093849388938A9568899E86C148F087C1C2
:106C980049F0120089806B6AB3EC3BF0CAC0A9F1D5
:106CA800CBC0AAF10101A951AA1105E0A9C1EAF0D6
:106CB800AAC1EBF01200A16BA26BA36BA46BA86B2B
:106CC800010EA76FAD6BCFD0AB6BAC6B1CD029ECB2
:106CD80053F00B500C1013E0AD0E0B6E010E0C6E42
:106CE800B8EC4AF00101A66F000E7224D96EDA6A78
:106CF800030EDA22A6C1DFFF722AAB4BAC2B0101CF
:106D0800ADAB81AC04D0ACBFE2D7AC05E0E3ABC11E
:106D1800ECF0ACC1EDF0000E0001EDBFFF0EEE6F20
:106D2800EF6FEC510101A1270001ED510101A223F0
:106D38000001EE510101A3230001EF510101A42339
:106D48007350140D0F0EF324D96E010EF420DA6E71
:106D5800DE50A15DDE50A259DE50A359DE50A45981
:106D680002E3A76BA86BADAB02D0A76BA86B81BC85
:106D780002D0A76BA86BACBF02D0AC0519E2000E1D
:106D880072240B6E0C6A030E0C22FF0E7224D96E4D
:106D9800DA6A020EDA22DF500D6E0E6A72500008AF
:106DA8000F6E000ED8A0E82A0108106E19EC41F009
:106DB8007350140D070EF324D96E010EF420DA6E09
:106DC80078C1F1F079C1F2F07AC1F3F00001F06B0B
:106DD800000EF025F46F010EF121F56F000EF2217F
:106DE800F66F000EF321F76FDE50F4191BE1DE5049
:106DF800F51918E1DE50F61915E1DE50F71912E120
:106E080001C3B1F103C3B0F105C3AFF107C3AEF1DC
:106E1800AEC10EF0AFC10FF0B0C110F0B1C111F0AA
:106E2800F8EC4EF097EC4DF0E1510101A56FA5513A
:106E38001AE0010E6B6E7350140D130EF324D96E05
:106E4800010EF420DA6E7350140D130EF324E16E64
:106E5800010EF420E26EE7500409DF6E6BC0EAF021
:106E68000001EB6B1200A751A81101E02DD782A4F5
:106E780002D0010E6B6E89900001EA6BEB6B120079
:106E880081A604D0230E486EFE0E03D0B60E486EBF
:106E9800FF0E496E81AA04D0230E4A6EFE0E03D05F
:106EA800B10E4A6EFF0E4B6E81A804D0230E4C6EB5
:106EB800FE0E03D0BB0E4C6EFF0E4D6E81AE04D09D
:106EC800230E4E6EFE0E03D0C00E4E6EFF0E4F6E9A
:106ED80081AC04D0230E506EFE0E03D0AC0E506E63
:106EE800FF0E516E81A404D0230E526EFE0E03D005
:106EF800CA0E526EFF0E536E81A204D0230E546E3A
:106F0800FE0E03D0CF0E546EFF0E556E81A004D036
:106F1800230E566EFE0E03D0C50E566EFF0E576E2C
:106F280083AE04D0230E586EFE0E03D0F90E586EB1
:106F3800FF0E596E83AC04D0230E5A6EFE0E03D09A
:106F4800F60E5A6EFF0E5B6E83AA04D0230E5C6E9B
:106F5800FE0E03D0F30E5C6EFF0E5D6E83A804D0A8
:106F6800230E5E6EFE0E03D0F00E5E6EFF0E5F6E99
:106F780083A604D0230E606EFE0E03D0ED0E606E65
:106F8800FF0E616E83A404D0230E626EFE0E03D042
:106F9800EA0E626EFF0E636E83A204D0230E646E47
:106FA800FE0E03D0E70E646EFF0E656E83A004D05C
:106FB800230E666EFE0E03D0E40E666EFF0E676E3D
:106FC800FA0E0001806FFA0E816F831C826F836B4B
:106FD80081CF84F0856B66C086F067C087F064C097
:106FE80088F065C089F062C08AF063C08BF060C029
:106FF8008CF061C08DF05EC08EF05FC08FF05CC019
:1070080090F05DC091F05AC092F05BC093F058C008
:1070180094F059C095F056C096F057C097F054C0F8
:1070280098F055C099F052C09AF053C09BF050C0E8
:107038009CF051C09DF04EC09EF04FC09FF04CC0D8
:10704800A0F04DC0A1F04AC0A2F04BC0A3F048C0C8
:10705800A4F049C0A5F0DDEF52F0636E0001A7511E
:1070680002E0EBEC3DF0626A0001A65101E1C8D0F4
:10707800040E631803E0140E631809E10101926B12
:10708800846B856B0001A76B070EA66F070C3F0E7C
:10709800631807E1FC6B0101926B0001A66BA76BFB
:1070A80012005F0E631807E10101936B926B0001F8
:1070B800A66BA76B12003F0E636406D05F0E636079
:1070C80003D0400E6318F0E1400E631808E1010E8A
:1070D8000101936F926B0001A66BA76B1200200E43
:1070E80063180CE1010EFC6F0101926B830E000125
:1070F800806FFF0E816FDDEC52F0EDD7650E6318DF
:1071080007E1FC5105E00101846B856B010E29D074
:107118006E0E631803E1020E0101926F700E631880
:1071280007E10101935104E0846B856B030E926FB4
:10713800700E631809E10001FC5106E08980010125
:10714800846B856B040E0DD0720E631859E1000133
:10715800FC5156E089801C0E0101856F2A0E846F50
:10716800050E926FB8D7635002EC14F0626E5AD0D5
:107178008980635038EC4DF0626E0101926B52D0F9
:107188008980340E0B6E0A0E0C6E0E6A0D6A010EA3
:10719800106E0F6A19EC41F00101FA832AEE34F0FF
:1071A8006BC0DFFF520E0001806FFD0E816F000E75
:1071B800836F010E826FDDEC52F0340E486E0A0EBA
:1071C800496E000E4B6E010E4A6E600E4C6EFF0E3D
:1071D8004D6E3BEC32F0496A010E486E56EC35F0C4
:1071E800FA93080EC9D78990626A1CD0080E6318F2
:1071F80019E18990626A6B6A926B846B856B12D015
:1072080001019251606E616A61500CE160500AE0C0
:10721800010AA9E0030AACE0010AB2E0070AE3E0C8
:10722800010AE4E062C0A6F00001A76B12007350E7
:10723800070D520EF324D96E010EF420DA6EDF2A00
:107248007350070D520EF324D96E010EF420DA6E36
:107258000F0EDF642FD07350070D520EF324D96E32
:10726800010EF420DA6EDF6A7350070D510EF32415
:10727800D96E010EF420DA6EDF2A7350070D510E15
:10728800F324D96E010EF420DA6E010EDF6412D0F9
:107298007350070D510EF324D96E010EF420DA6EE7
:1072A800DF6A7350070D500EF324D96E010EF420D7
:1072B800DA6EDF2A7350070D520EF324D96E010ED1
:1072C800F420DA6EDF500001CA6FCAC0CBF0CC6B75
:1072D800CD6BCE6BCDC0CEF0CCC0CDF0CBC0CCF05A
:1072E800CB6B7350070D510EF324D96E010EF420A9
:1072F800DA6EDF50CF6FCFC0D0F0D16BD26BD36BCB
:107308000C0ED890D037D137D237D337E82EF9D7EB
:107318007350070D500EF324D96E010EF420DA6E67
:10732800DF50D46FD4C0D5F0D66BD76BD86B0D0EA9
:10733800D890D537D637D737D837E82EF9D7D051A0
:10734800D525D96FD151D621DA6FD251D721DB6F2C
:10735800D351D821DC6FCB51D925DD6FCC51DA213F
:10736800DE6FCD51DB21DF6FCE51DC21E06F735032
:10737800070D530EF324D96E010EF420DA6EDDC02A
:10738800DEFFDEC0DEFFDFC0DEFFE0C0DEFF7350E1
:10739800200D000EF324A36F020EF420A46F735087
:1073A800070D530EF324D96E010EF420DA6EDECFEA
:1073B800A5F0DECFA6F0DECFA7F0DECFA8F063EC15
:1073C8000EF06A6E6A5019E07E0E806FFC0E816FB7
:1073D8007350070D530EF324D96E010EF420DA6EA4
:1073E800DECF82F0DECF83F0DECF84F0DECF85F013
:1073F8006AC086F0876BDDEC52F001019F6B1200CA
:10740800FA83340E0B6E0A0E0C6E0E6A0D6A010EAC
:10741800106E0F6A19EC41F02AEE34F073C0DFFFEA
:10742800FF0EE8CF35FA7350140D130EF324D96EFE
:10743800010EF420DA6EDFA403D0010EE8CF38FA8B
:107448007350140D130EF324D96E010EF420DA6E66
:10745800DFA003D0020EE8CF3AFA7350140D130ED2
:10746800F324D96E010EF420DA6EDFA203D0020EE7
:10747800E8CF3AFA82A403D0080EE8CF3AFA506A65
:10748800516ABB0E0001806FFB0E816FCFCF82F077
:10749800836BCECF84F0856B50C086F051C087F0E7
:1074A800360E5024D96E0A0E5120DA6EDF50886FDE
:1074B800896BDDEC52F06C0E5024D96E010E512010
:1074C800DA6EDF1C4F6E360E5024D96E0A0E51202C
:1074D800DA6E360E5024E16E0A0E5120E26EE75045
:1074E8004F14DF6E590E0001806FFF0E816F360E4C
:1074F8005024D96E0A0E5120DA6EDF50826F836BEA
:10750800DDEC52F0504A512A51BEBBD7515003E12D
:10751800070E505CB6E37350140D130EF324D96EA6
:10752800010EF420DA6EDF506B6E7350140D010EED
:10753800F324D96E010EF420DA6EDF504E6E4EC081
:107548003FFA7350140D020EF324D96E010EF42085
:10755800DA6EDF504E6E4EC040FA7350140D030EB3
:10756800F324D96E010EF420DA6EDF504E6E4EC051
:1075780041FA7350140D040EF324D96E010EF42051
:10758800DA6EDF504E6E4EC042FA7350140D050E7F
:10759800F324D96E010EF420DA6EDF504E6E4EC021
:1075A80043FA7350140D060EF324D96E010EF4201D
:1075B800DA6EDF504E6E4EC044FA496A140E486EB9
:1075C80056EC35F0FA93899012000001BD6B010E5C
:1075D800BC6F8980BBD07350200D000EF324626EFF
:1075E800020EF420636E340E646E0A0E656E010E90
:1075F800676E666ABE0E686E696A4DEC11F073506C
:10760800070D530EF324D96E010EF420DA6E78C1FB
:10761800B1F079C1B2F07AC1B3F00001B06B000EDD
:10762800B025B46F010EB121B56F000EB221B66F4F
:10763800000EB321B76FDE50B4192CE1DE50B51936
:1076480029E1DE50B61926E1DE50B71923E16FECC7
:107658004CF00FC0C0F010C0C1F011C0C2F012C091
:10766800C3F0000EE8CF34FA2AEE35F0C3C0DFFFCE
:10767800E8CF36FA2AEE37F0C2C0DFFFE8CF38FA93
:107688002AEE39F0C1C0DFFFE8CF3AFA2AEE3BF024
:10769800C0C0DFFF0101FA93BEC048F0BFC049F087
:1076A80056EC35F048C0BAF049C0BBF081AC53D0B5
:1076B8000001BE51BA1903E1BF51BB190BE0F80E26
:1076C800806FFE0E816FBAC082F0BBC083F0DDEC24
:1076D80052F041D086EC52F029EC53F00B500C10CC
:1076E80004E0010E01019F6F36D00001B96B050E51
:1076F800B86F1CD00B0E0001AC6F620EE82EFED7DF
:10770800AC2FFCD700F029EC53F00B500C100EE016
:107718000001BC6BBD6BF70E806FFD0E816FB8C0AA
:1077280082F0B9C083F0DDEC52F008D00001B80750
:10773800D8A0B907B829DEE1B929DCE129EC53F072
:107748000B500C1003E00001BC6BBD6B0001BC5179
:10775800BD1101E040D701019F6B89901200735061
:10776800140D070EF324D96E010EF420DA6EDECF65
:10777800DCF0DECFDDF0DECFDEF0DECFDFF0735001
:10778800140D070EF324D96E010EF420DA6E73502F
:10779800140D0B0EF324E16E010EF420E26EDE50A0
:1077A800E65CDE50E658DE50E658DE50E65815E254
:1077B800010E6B6E7350140D130EF324D96E010E67
:1077C800F420DA6E7350140D130EF324E16E010EDB
:1077D800F420E26EE7500409DF6E7350140D0F0EAB
:1077E800F324D96E010EF420DA6EDECFCCF0DECFB2
:1077F800CDF0DECFCEF0DECFCFF07350140D070EF4
:10780800F324D96E010EF420DA6EDECFD0F0DECF8D
:10781800D1F0DECFD2F0DECFD3F00001CC51D025AD
:10782800D46FCD51D121D56FCE51D221D66FCF5142
:10783800D321D76F7350140D0B0EF324D96E010E9C
:10784800F420DA6ED451DE5CD551DE58D651DE58BC
:10785800D751DE5815E2010E6B6E7350140D130EDE
:10786800F324D96E010EF420DA6E7350140D130E42
:10787800F324E16E010EF420E26EE7500409DF6E96
:107888006B6A7350200D000EF324A36F020EF420D0
:10789800A46FDCC0A5F0DDC0A6F0DEC0A7F0DFC095
:1078A800A8F063EC0EF0E06FE05115E0010E6B6E8E
:1078B8007350140D130EF324D96E010EF420DA6EF2
:1078C8007350140D130EF324E16E010EF420E26ED2
:1078D800E7500409DF6E6BC0CAF0CB6B12001B6E59
:1078E8001B5001E0010C74A202D074501200000E6B
:1078F800A1EC52F00A0E266E03D016EC53F02606C1
:107908002650FBE1236A000E146A156A166A176A84
:1079180012EC51F0E80601E097D0AA0E146E010EA1
:10792800156E166A176A080E12EC51F0E80651E156
:10793800266A26501C0FD96EDA6A16EC53F0DF6EF1
:10794800262A030E2664F5D71E047EE1AA0E1F1808
:107958007BE1030E256EE80E246E15D0146A156AB5
:10796800166A400E176EA90E12EC51F000090EE0CF
:107978000B0E1A6E620EE82EFED71A2EFCD700D018
:107988002406D8A0250624502510E8E12450251007
:107998005BE0146A156A166A176A3A0E12EC51F01F
:1079A800000952E1266A26501C0FD96EDA6A16ECD5
:1079B80053F0DF6E262A030E2664F5D71CBC03D0CD
:1079C800216A040E02D0216A0C0E206E20C023F01A
:1079D8003BD0146A156A166A176AA90E12EC51F0A0
:1079E8001A6E020E1A6003D0236EA90E02D0010E81
:1079F800236E226E030E256EE80E246E14D0146AD0
:107A0800156A166A176A225012EC51F000090EE046
:107A18000B0E1A6E620EE82EFED71A2EFCD700D077
:107A28002406D8A0250624502510E9E12450251065
:107A38000AE0146A020E156E166A176A100E12EC26
:107A480051F0000901E0236A23C06EF02EEC53F0D8
:107A5800235001E14AD7749048D7BEC0F6FFBFC093
:107A6800F7FF000EF86E0F0EF76403D00800F5500C
:107A780005D0F6CFE9FFF7CFEAFFEF502F0A13E062
:107A8800BEC0F6FFBFC0F7FF000EF86E0F0EF7641A
:107A980003D00800F55005D0F6CFE9FFF7CFEAFF8D
:107AA800EF505C0A03E10001BE4BBF2B000120EE42
:107AB80006F0BC51D926BD51DA22DE6ADE6ADE6ADA
:107AC800DD6ABEC0F6FFBFC0F7FF000EF86E0F0EEE
:107AD800F76403D00800F55005D0F6CFE9FFF7CFDB
:107AE800EAFFEF506A6E200E6A6012D0BCC062F0E6
:107AF800BDC063F0656A646A7EEC2EF0C36F20EE49
:107B080012F0BC51D926BD51DA22DE6ADD6A5DD099
:107B1800BCC013F0BDC014F0BE0E156ECFEC2BF038
:107B28000001C36FC35151E1BCC0B6F0BDC0B7F08E
:107B380024EC47F0C36F20EE14F0BC51D926BD5198
:107B4800DA2210EE0BF0DE50E126DD50E222E7509B
:107B5800C26FC35108E0040EC31937E1C2B535D06E
:107B6800050EC36F32D0C2B530D020EE12F0BC5132
:107B7800D926BD51DA22DECFC0F0DDCFC1F020EE2C
:107B88000BF0C051D926C151DA22DFA8E9D7BCC011
:107B9800D9FFBDC0DAFFDECF0BF0DDCF0CF0C0C0DF
:107BA8000DF0C1C00EF057EC48F0000120EE06F0D1
:107BB800BC51D926BD51DA220BC0DEFF0CC0DEFF56
:107BC8000DC0DEFF0EC0DEFFA3D7C3511200736ADB
:107BD800736A030E736401D0A0D07350140D130E92
:107BE800F324D96E010EF420DA6EDF6A7350140D97
:107BF800000EF324D96E010EF420DA6EDF6A73509A
:107C0800140D070EF324D96E010EF420DA6EDE6A25
:107C1800DE6ADE6ADD6AF3C148F0496A4A6A4B6A7D
:107C28004AC04BF049C04AF048C049F0486AF2C11E
:107C38004CF04D6A4E6A4F6A4DC04FF04CC04EF042
:107C48004D6A4C6AF1C150F0516A526A536A50C089
:107C580053F0526A516A506A0101F0515024546E2F
:107C6800000E5120556E000E5220566E000E532005
:107C7800576E4C505424586E4D505520596E4E50E6
:107C880056205A6E4F5057205B6E485058245C6EF1
:107C9800495059205D6E4A505A205E6E4B505B2009
:107CA8005F6E7350140D0B0EF324D96E010EF42081
:107CB800DA6E5CC0DEFF5DC0DEFF5EC0DEFF5FC067
:107CC800DEFF9B0E0001806FFB0E816F73C082F098
:107CD800836B7350140D0B0EF324D96E010EF42030
:107CE800DA6EDECF84F0DECF85F0DECF86F0DECF31
:107CF80087F07350140D0B0EF324D96E010EF42087
:107D0800DA6EDECF88F0DECF89F0DECF8AF0DECF04
:107D18008BF0DDEC52F0732A5CD70101936B000104
:107D2800FC6B0101926B846B856B020E6B6E899004
:107D3800020C0600D9CF05F0DACF06F0F2A01CD06D
:107D480081BC02D08994899281A802D089A20FD0DF
:107D58009380939424EE04F0010EDBBE07D0000E4E
:107D6800DE5C020EDE5802E3939201D0938281B862
:107D780089B201D09384F290F2B281B079D081B8FF
:107D880089B29392831C086E811C076E04C409F0A3
:107D980005C40AF00ABE03D0020E0A5C2BE2094AA7
:107DA8000A2A09C004F40AC005F402C409F003C48D
:107DB8000AF0060E0924D96E040E0A20DA6E08C0ED
:107DC800DFFF060E0924D96E060E0A20DA6E07C0F8
:107DD800DFFF094A0A2A0168010E026E09C003F092
:107DE8000AC004F0015003160250041603C002F43E
:107DF80004C003F481B889B29384938481A0FED728
:107E080081A802D089A202D0939401D0938424EE51
:107E180004F0010EDBBE05D0000EDE5C020EDE585B
:107E280003E201019C5102E0939201D0938207A8DA
:107E38001ED00BD0898202D0898405D0899417D0AE
:107E480089A215D08994899212D00850016E026ACD
:107E580002500DE10150040AF3E0100AF1E0340A7F
:107E6800E9E01F0AF0E07F0AE7E01F0AE7E0F29284
:107E780006C0DAFF05C0D9FF75921100326A20EEFC
:107E880004F02450D9262550DA22DF5001E197D09A
:107E980020EE2AF02450D9262550DA22DECF35F0FC
:107EA800DECF36F0DECF37F0DECF38F02E0E2424CA
:107EB8001A6E000E25201B6E35C01CF036C01DF052
:107EC80037C01EF038C01FF0216A010E206E20EE68
:107ED80001F02450D9262550DA22DF50DBEC45F09A
:107EE800000903E0010E326E6AD020EE04F024503F
:107EF800D9262550DA22DF6A20EE16F02450D9263A
:107F08002550DA2210EE1EF02450E1262550E222F8
:107F1800E6CF2AF0E6CF2BF0E6CF2CF0E6CF2DF017
:107F28002A50355C2E6E2B5036582F6E2C503758F1
:107F3800306E2D503858316EDE502E5CDE502F5882
:107F4800DE503058DE5031583AE220EE03F024502B
:107F5800D9262550DA22DF50336E346A345003E1D3
:107F6800020E335C2CE320EE16F02450D92625505F
:107F7800DA22DE503526DE503622DE503722DD503A
:107F880038222E0E24241A6E000E25201B6E35C0B2
:107F98001CF036C01DF037C01EF038C01FF0216A33
:107FA800010E206E20EE01F02450D9262550DA2249
:107FB800DF50DBEC45F03306D8A03406CFD732507B
:107FC80012007350070D520EF324D96E010EF420DF
:107FD800DA6EDF500001CA6FCAC0CBF0CC6BCD6B34
:107FE800CE6BCDC0CEF0CCC0CDF0CBC0CCF0CB6B3F
:107FF8007350070D510EF324D96E010EF420DA6E7A
:10800800DF50CF6FCFC0D0F0D16BD26BD36B0C0EDB
:10801800D890D037D137D237D337E82EF9D7735025
:10802800070D500EF324D96E010EF420DA6EDF50DE
:10803800D46FD4C0D5F0D66BD76BD86B0D0ED89053
:10804800D537D637D737D837E82EF9D7D051D525F1
:10805800D96FD151D621DA6FD251D721DB6FD351E5
:10806800D821DC6FCB51D925DE6FCC51DA21DF6FF7
:10807800CD51DB21E06FCE51DC21E16F7350200D33
:10808800000EF324A36F020EF420A46FDEC0A5F047
:10809800DFC0A6F0E0C0A7F0E1C0A8F063EC0EF0E6
:1080A800DD6FDD5118E0DB0E806FFB0E816F73C052
:1080B80082F0836BDEC084F0DFC085F0E0C086F01C
:1080C800E1C087F0DDC088F0896BDDEC52F0010E6D
:1080D80001019F6F12D07350070D530EF324D96E10
:1080E800010EF420DA6EDEC0DEFFDFC0DEFFE0C086
:1080F800DEFFE1C0DEFF01019F6B899012002F6C4B
:10810800696664617461302E62696E20002F6C6943
:108118006664617461312E62696E20002F6C696635
:1081280064617461322E62696E20002F6C69666426
:10813800617461332E62696E20002F6C6966646118
:108148007461342E62696E20002F6C6966646174F4
:1081580061352E62696E20002F6C696664617461F6
:10816800362E62696E20002F6C696664617461370F
:108178002E62696E20002F6C696664617461382E06
:1081880062696E20002F6C696664617461392E62C1
:10819800696E20002F6C696664617461612E626982
:1081A8006E20002F6C696664617461622E62696E6C
:1081B80020002F6C696664617461632E62696E20A9
:1081C800002F6C696664617461642E62696E2000B8
:1081D8002F6C696664617461652E62696E20002F78
:1081E8006C696664617461662E62696E20000000C5
:1081F8000000000000000000000000000000000077
:108208000000000000000000000000000000000066
:108218000000000000000000000000000000000056
:10822800000000000000000000000BC015F00CC0AA
:1082380016F00F50101001E1120015C0D9FF16C03A
:10824800DAFF0DC0DFFF0F501524116E10501620F5
:10825800126EFF0E1124D96EFF0E1220DA6E0DC0B9
:10826800DFFF105004E1030E0F5C01E2120020EE64
:1082780001F01550D9261650DA220DC0DFFF20EE86
:1082880002F01550D9261650DA220DC0DFFF0F5024
:108298001524116E10501620126EFE0E1124D96E80
:1082A800FF0E1220DA6E0DC0DFFF0F501524116E7D
:1082B80010501620126EFD0E1124D96EFF0E1220DA
:1082C800DA6E0DC0DFFF105004E1070E0F5C01E20B
:1082D800120020EE03F01550D9261650DA220DC0F0
:1082E800DFFF0F501524116E10501620126EFC0E71
:1082F8001124D96EFF0E1220DA6E0DC0DFFF105068
:1083080004E1090E0F5C01E2120015C011F016C05D
:1083180012F0111E121E114A122A030E1114136EA6
:10832800146A135015261450162213500F5E145059
:10833800105AFC0E0F160BD015C0D9FF16C0DAFF65
:108348000DC0DFFF0F06D8A01006154A162A0F50D9
:108358001010F2E112000001915190118F1103E108
:10836800020E8E5D0FE320EE12F08C51D9268D514E
:10837800DA22DE508E5DDE508F59DE509059DE5085
:10838800915902E3020E2CD0966B6AD08CC044F04F
:108398008DC045F08EC046F08FC047F090C048F0C1
:1083A80091C049F028EC1BF044C097F045C098F004
:1083B80046C099F047C09AF0000197519811991159
:1083C8009A115DE09705981199119A11DBE09729A8
:1083D80009E1982907E1992905E19A2903E1010EA4
:1083E800966F4DD08CC044F08DC045F08EC046F0DD
:1083F8008FC047F090C048F091C049F04A6A4B6A74
:108408004C6A4D6ACBEC18F0966F965138E120EE25
:108418000EF08C51D9268D51DA22DE2806E1DE28AD
:1084280004E1DE2802E1DE2813E020EE0EF08C5194
:10843800D9268D51DA22DE2A000EDE22DE22DE2245
:1084480020EE05F08C51D9268D51DA22000EDB8002
:1084580097C08EF098C08FF099C090F09AC091F0B4
:1084680020EE12F08C51D9268D51DA22DE508E5D25
:10847800DE508F59DE509059DE50915987E396515E
:108488001200136814680B50D96EDA6ADE50DE10D9
:1084980001E181D00B50D96EDA6ADECF17F0DDCF5B
:1084A80018F002D0174A182A17C0F6FF18C0F7FFAD
:1084B800000EF86E0F0EF76403D00800F55005D0D3
:1084C800F6CFE9FFF7CFEAFFEF500D6E200E0D64EF
:1084D80013D017C0F6FF18C0F7FF000EF86E0F0E86
:1084E800F76403D00800F55005D0F6CFE9FFF7CFC1
:1084F800EAFFEF503A0AD6E117C0F6FF18C0F7FFB7
:10850800000EF86E0F0EF76403D00800F55005D082
:10851800F6CFE9FFF7CFEAFFEF503A0A41E10B50F7
:10852800D96EDA6ADECF11F0DDCF12F011C0F6FF96
:1085380012C0F7FF000EF86E0F0EF76403D00800A4
:10854800F55005D0F6CFE9FFF7CFEAFFEF500D6EF3
:10855800D00E0D24156E166AFF0E1622114A122A25
:10856800165019E10A0E155C16E21750111813E19E
:108578001850121810E1155016100DE115C013F01F
:1085880016C014F0174A182A0B50D96EDA6A17C0A9
:10859800DEFF18C0DDFF13C00BF014C00CF0120092
:1085A800136A146AF8D789800001EE6BEF6BC6EC8A
:1085B8004DF015C0F0F016C0F1F00001F1BF0AD07F
:1085C800040EF15D07E3000EF025EE6FFC0EF121BD
:1085D800EF6F04D0F0C0EEF0F1C0EFF07350070D6C
:1085E800530EF324D96E010EF420DA6E78C1E6F04A
:1085F80079C1E7F07AC1E8F0E56B000EE525E96F8F
:10860800010EE621EA6F000EE721EB6F000EE8216C
:10861800EC6FDE50E9191BE1DE50EA1918E1DE5073
:10862800EB1915E1DE50EC1912E101C3F5F003C3B3
:10863800F4F005C3F3F007C3F2F0F2C00EF0F3C094
:108648000FF0F4C010F0F5C011F0F8EC4EF082B461
:1086580015D07350200D000EF3240001A36F020EF5
:10866800F420A46F000EA56F030EA66F010EA86F6D
:10867800A76BEE0EA96FF5EC0AF0ED6F0001ED5156
:1086880009E0070E806FFE0E816FEDC082F0836BEC
:10869800DDEC52F01BEC39F09F6B8990960E0001CF
:1086A800806FFD0E816FCFCF82F0836BCECF84F0C9
:1086B800856BDDEF52F0020E0D5E000E0E5A0F5A5A
:1086C800105A20EE12F00B50D9260C50DA22FE0E6A
:1086D800DE24116EFF0EDE20126EFF0EDE20136EFA
:1086E800FF0EDE20146E11500D5C12500E58135000
:1086F8000F581450105805E30B6A0C6A0D6A0E6A7D
:10870800120020EE26F00B50D9260C50DA22DECFCC
:1087180011F0DECF12F0DECF13F0DECF14F020EE32
:1087280002F00B50D9260C50DA22DF50156E15C016
:1087380016F0176A186A196A16500D02F3CF1AF064
:10874800F4CF1BF01C6A1D6A0E02F3501B26F4506E
:108758001C22000E1D2217500D02F3501B26F45048
:108768001C22000E1D2216500F02F3501C26F45036
:108778001D2217500E02F3501C26F4501D221850CB
:108788000D02F3501C26F4501D2210501602F3500F
:108798001D2617500F02F3501D2618500E02F350D5
:1087A8001D2619500D02F3501D2611501A240B6E68
:1087B80012501B200C6E13501C200D6E14501D20DF
:1087C8000E6E1200FBC14AF070D066EC52F04A6E91
:1087D800FB1978E0150E496E4B0E486EBE0EE82E5A
:1087E800FED7482EFCD7492EFAD700D06BD021EC03
:1087F8004EF04B6E4B5066E04BB06D2A4BB26D0697
:108808000F0E6D16000E0B6EC00E99EC4FF055EC66
:1088180052F0000E0B6EC00E99EC4FF06D500F0D1C
:10882800340EF3240F6E0C0EF420106E84EC4BF013
:108838000D0E496E2D0E486ED80EE82EFED7482E26
:10884800FCD7492EFAD74BA43DD00C6A0B6A6DC0F1
:108858000DF0BDEC50F02D0E0001806FFD0E816F04
:108868006DC082F0836BDDEC52F06DC04AF0000EF3
:108878000B6E800E99EC4FF055EC52F0000E0B6E1B
:10888800800E99EC4FF06D500F0D340EF3240F6EDF
:108898000C0EF420106E84EC4BF0000E0B6EC00E24
:1088A80099EC4FF055EC52F00DD001019851486EFB
:1088B800496A495007E14850010A87E0030A85E000
:1088C800010A95E04A5012001F6A206A186A196A5C
:1088D80001D0122A010E1E6E1250D96EDA6A200ECD
:1088E800DE1813E0F70E146E15681250D96EDA6AA6
:1088F800DF50166E176A1450162615501722175097
:1089080003E1050E165C01E31E6A1EC01AF01B6A1D
:108918001A501B1006E0DDD7196A010E186E122ACC
:1089280025D01250D96EDA6ADF50146E156A1550C8
:108938001DE114502B0AF3E0060AEEE017D00A0EE8
:108948001F02F3CF14F0F4CF15F02002F3501526D0
:108958001250D96EDA6ADF50145E000E155A300EC6
:1089680014241F6E000E1520206ED9D7D00E146E59
:1089780015681250D96EDA6ADF50166E176A1450ED
:10898800162615501722175005E10A0E165C02E24A
:10899800010E01D0000E1C6E1D6A1C501D10CFE187
:1089A800185019100DE11FC014F020C015F0141E46
:1089B800151E144A152A14C012F015C013F012001F
:1089C8001FC012F020C013F012000001EF6B898065
:1089D80070D0C6EC4DF015C0EDF016C0EEF00001F9
:1089E800EEBF06D0040EEE5D03E3010EEF6F03D079
:1089F800F2C0F0F0F16B82B414D07350200D000E69
:108A0800F324A36F020EF420A46F000EA56F030ECB
:108A1800A66F010EA86FA76BF00EA96FF5EC0AF010
:108A2800F26FF25109E0070E806FFE0E816FF2C0FF
:108A380082F0836BDDEC52F07350070D530EF32474
:108A4800D96E010EF420DA6E78C1E6F079C1E7F04C
:108A58007AC1E8F00001E56B000EE525E96F010E2B
:108A6800E621EA6F000EE721EB6F000EE821EC6FBC
:108A7800DE50E9191BE1DE50EA1918E1DE50EB1966
:108A880015E1DE50EC1912E101C3F6F003C3F5F06D
:108A980005C3F4F007C3F3F0F3C00EF0F4C00FF011
:108AA800F5C010F0F6C011F0F8EC4EF01BEC39F000
:108AB8009F6B0001EF518DE0899012008980000EB4
:108AC8000B6E030E0C6E0E6AF60E0D6E010E106E16
:108AD8000F6A19EC41F0AB0E0001806FFE0E816F3A
:108AE800DDEC52F00001E66BE76B2E0EE7EC52F07E
:108AF80082B415D07350200D000EF3240001A36F2B
:108B0800020EF420A46F000EA56F030EA66F010ECF
:108B1800A86FA76BE30EA96FF5EC0AF0E56F0001EB
:108B2800E55109E07C0E806FFF0E816FE5C082F091
:108B3800836BDDEF52F029EC53F00B500C1027E05B
:108B4800E80E0B6E0C6AB8EC4AF00001E26FE851CF
:108B5800100B0B6E000E0C6EE25120EC25F00BC0D2
:108B6800E9F00CC0EAF0040E0001E919EA1102E18B
:108B7800AAEC51F0020E0001E919EA1102E173ECC6
:108B88004FF00001E905EA1102E1E5EC3FF00001D0
:108B9800E64BE72BE75103E1C80EE65DA6E3240E9A
:108BA800806FFF0E816FDDEC52F089901200236E0A
:108BB8002350D8A4040C2050211001E1040C74B0F7
:108BC800030C74B4020C6EB608D0090ED8901C368B
:108BD8001D361E361F36E82EF9D7200421101AE15B
:108BE8001CC014F01DC015F01EC016F01FC017F0F1
:108BF800180E12EC51F0000945E11AC00DF01BC027
:108C08000EF0FE0E0F6EA4EC4EF000093BE0206A59
:108C1800216A38D06EC022F0060E221609E020C064
:108C280014F021C015F0166A176A970E12EC51F06D
:108C38001CC014F01DC015F01EC016F01FC017F0A0
:108C4800190E12EC51F000091DE11AC00DF01BC0FD
:108C58000EF0FC0E0F6EA4EC4EF0000908E0020EB8
:108C68001B262006D8A0210620502110EEE10D6A0F
:108C78000E6AFD0E0F6EA4EC4EF0000903E1216AA6
:108C8800010E206E2EEC53F020502110D8A4010CB8
:108C9800000C0F0EC16E969496929690929A090EB9
:108CA800106E1E0E0F6EE40EE82EFED70F2EFCD7A8
:108CB800102EFAD700D0090E106E1E0E0F6EE40E9D
:108CC800E82EFED70F2EFCD7102EFAD700D0D00EE4
:108CD8000F6ECA0EE82EFED70F2EFCD7000E0B6EB5
:108CE800300E99EC4FF0150E0F6EC60EE82EFED71B
:108CF8000F2EFCD700D0000E0B6E300E99EC4FF003
:108D0800000E0B6E300E99EC4FF0000E0B6E390E04
:108D180099EC4FF0000E0B6E140E99EC4FF0000E0C
:108D28000B6E560E99EC4FF0000E0B6E6D0E99EC13
:108D38004FF0000E0B6E700E99EC4FF0000E0B6E9C
:108D48000C0E99EC4FF0000E0B6E060E99EC4FF0DE
:108D5800000E0B6E010E99EC4FF0680E0F6EE40ECC
:108D6800E82EFED70F2EFCD700D01200060EF66EA6
:108D7800810EF76E000EF86E0CEE34F011EE2CF04A
:108D88000900F5CFEEFFE550E150FAE1E250F8E1D5
:108D9800F50EF66EA50EF76E000EF86E02EEA0F058
:108DA80010EE13F00900F5CFEEFFE550E150FAE1BF
:108DB800E20EF66EA50EF76E000EF86E01EEE7F005
:108DC80010EE13F00900F5CFEEFFE550E150FAE19F
:108DD800800EF66EA60EF76E000EF86E0900F5CF3F
:108DE80074F004EE00F018EE34F0EE6AE550E1504D
:108DF800FCE1E250FAE103EE00F011EE00F0EE6A59
:108E0800E550E150FCE1E250FAE102EE00F0A00E7C
:108E1800EE6AE806FDE101EE00F0A10EEE6AE80652
:108E2800FDE10001FC6B00EE6BF0090EEE6AE8064E
:108E3800FDE175907592000EF86E000149EF07F09C
:108E4800B6C062F0B7C063F0656A646A7EEC2EF063
:108E5800BB6FBB5102E0BB511200B6C0D9FFB7C00F
:108E6800DAFFDECF39F0DDCF3AF020EE0EF0B65162
:108E7800D926B751DA22DECF3BF0DECF3CF0DECF89
:108E88003DF0DECF3EF0FEEC48F00001BB6FBB5179
:108E9800E2E120EE12F0B651D926B751DA22DECF40
:108EA800B9F0DDCFBAF0B9C0D9FFBAC0DAFFDF50E8
:108EB800B86FB85103E1040EBB6FCDD720EE0BF0AD
:108EC800B951D926BA51DA22DFB616D0B9C00BF09B
:108ED800BAC00CF020EE14F0B651D926B751DA22F8
:108EE800DECF0DF0DDCF0EF0106A0B0E0F6EF4EC36
:108EF8004DF00B500C10AFE0B6C0A3F0B7C0A4F013
:108F0800A66BA56B5CEC21F00001BB6FBB51A3E124
:108F1800A4D7B6C062F0B7C063F0656A646A7EEC35
:108F28002EF0BF6FBF5157E1BD6BBE6BB6C0D9FF06
:108F3800B7C0DAFFDECF39F0DDCF3AF020EE0EF021
:108F4800B651D926B751DA22DECF3BF0DECF3CF05E
:108F5800DECF3DF0DECF3EF0FEEC48F00001BF6F03
:108F6800BF5139E120EE12F0B651D926B751DA22B5
:108F7800DECFBAF0DDCFBBF0BAC0D9FFBBC0DAFF95
:108F8800E50EDE1810E020EE12F0B651D926B751E2
:108F9800DA22DECFBAF0DDCFBBF0BAC0D9FFBBC052
:108FA800DAFFDF5009E1BD4BBE2BB851BD1906E110
:108FB800B951BE1910E002D0BD6BBE6BB6C0A3F0AC
:108FC800B7C0A4F0A66B010EA56F5CEC21F0000100
:108FD800BF6FBF51ABE0040EBF1902E1070EBF6FB0
:108FE800BF511200C0C0B6F0C1C0B7F0B96B010ED6
:108FF800B86F8DEC47F06A6E6A5053E1C0C0D9FF74
:10900800C1C0DAFFDECF39F0DDCF3AF020EE0EF046
:10901800C051D926C151DA22DECF3BF0DECF3CF079
:10902800DECF3DF0DECF3EF0FEEC48F06A6E6A50CF
:1090380038E1000120EE12F0C051D926C151DA22E0
:10904800DECF0BF0DDCF0CF00E6A0D6A106A200E31
:109058000F6E2DEC52F0000120EE12F0C051D9260F
:10906800C151DA22DECF0BF0DDCF0CF020EE14F088
:10907800C051D926C151DA22DECF0DF0DDCF0EF076
:10908800106A0B0E0F6E62EC50F0C0C0D9FFC1C061
:10909800DAFF10EE04F0DE50E126DD50E222010E88
:1090A800E76E6A5012001A0E0D240F6E000E0E2085
:1090B800106E0F28D96E000E1020DA6EDF50126E77
:1090C800116A1A0E0D24D96E000E0E20DA6EDF50CA
:1090D800111211C017F012C018F0196A1A6A0BC0E1
:1090E800D9FF0CC0DAFF030EDE1829E1140E0D2497
:1090F8000F6E000E0E20106E0F28D96E000E102075
:10910800DA6EDF50126E116A140E0D24D96E000E3D
:109118000E20DA6EDF501110136E1250146E156A9D
:10912800166A14C016F013C015F0146A136A1350A7
:109138001712145018121550191216501A1217C077
:109148000BF018C00CF019C00DF01AC00EF0120088
:10915800226E2250D8A4040C2050211001E1040CE6
:1091680074B0030C6EB608D0090ED8901C361D36A4
:109178001E361F36E82EF9D7215006E1020E205C74
:1091880003E2246A110E02D0246A120E236E23C051
:1091980025F01CC014F01DC015F01EC016F01FC02D
:1091A80017F0255012EC51F000091DE11AC00BF020
:1091B8001BC00CF0020E0E6E0D6A4EEC4EF000094C
:1091C80008E0020E1B262006D8A0210620502110F8
:1091D800EDE1120E251807E1146A156A166A176A76
:1091E8000C0E12EC51F02EEC53F020502110D8A4A4
:1091F800010C000C436A20EE2AF03950D9263A5067
:10920800DA223B50DE1809E13C50DE1806E13D50F9
:10921800DE1803E13E50DE1839E039C024F03AC0C8
:1092280025F042EC3FF0436E435030E12E0E3924D6
:109238001A6E000E3A201B6E3BC01CF03CC01DF09D
:109248003DC01EF03EC01FF0216A010E206E20EEC8
:1092580001F03950D9263A50DA22DF50ACEC48F008
:10926800000906E03B683C683D683E68010E436EB5
:1092780020EE2AF03950D9263A50DA223BC0DEFFD8
:109288003CC0DEFF3DC0DEFF3EC0DEFF43501200A3
:10929800D4C0DAF0D5C0DBF0DA0E0B6E45EC42F044
:1092A8000BC0DCF00CC0DDF00001DDBF0B0CD8906A
:1092B800DC35D96EDD35DA6E8C0ED926010EDA2250
:1092C800DECFD8F0DDCFD9F0D851D91105E0D8C01C
:1092D800D9FFD9C0DAFFDF6AD251D31105E0D2C075
:1092E800D9FFD3C0DAFFDF6AD890DC35D96EDD3517
:1092F800DA6E8C0ED926010EDA22D2C0DEFFD3C078
:10930800DDFFD251D311D8B4000CD60501E0000C12
:10931800D20E666E676AD40E686E696A09EC00F050
:10932800D76FD751120003D00B4A0C2A0D2A0D50C3
:10933800D96EDA6ADF500E6E0BC0F6FF0CC0F7FF6D
:10934800000EF86E0F0EF76403D00800F55005D034
:10935800F6CFE9FFF7CFEAFFEF500E1813E10BC085
:10936800F6FF0CC0F7FF000EF86E0F0EF76403D07F
:109378000800F55005D0F6CFE9FFF7CFEAFFEF5028
:109388000009D2E10BC0F6FF0CC0F7FF000EF86E23
:109398000F0EF76403D00800F55005D0F6CFE9FFAB
:1093A800F7CFEAFFEF500E6E0D50D96EDA6ADF5034
:1093B8000E5C0B6E0C6AD8A00C0612007350140DCC
:1093C800070EF324D96E010EF420DA6E000EDE24A7
:1093D800CA6F010EDE20CB6F000EDE20CC6F000EB0
:1093E800DE20CD6F7350140D070EF324D96E010ED5
:1093F800F420DA6ECAC0DEFFCBC0DEFFCCC0DEFFD1
:10940800CDC0DEFF7350140D070EF324D96E010E84
:10941800F420DA6EDECFCEF0DDCFCFF07350200D22
:10942800000EF324A36F020EF420A46FCEC0A5F0A3
:10943800CFC0A6F0A76BA86B63EC0EF0D06FD0512D
:1094480003E0010E6B6E010C6B6A12000BC012F088
:109458000CC013F00DC014F00EC015F00F06D8A004
:1094680010060F280CE110280AE10B6A0C6A12009A
:10947800124A132A144A152A0F06D8A0100612C039
:10948800F6FF13C0F7FF0800F55015E014C0D9FF28
:1094980015C0DAFFDF500FE00F5010100CE014C0B9
:1094A800D9FF15C0DAFF12C0F6FF13C0F7FFDE5070
:1094B8000900F518DDE012C0F6FF13C0F7FF080039
:1094C800F5CF11F014C0D9FF15C0DAFFDF50115CD9
:1094D8000B6E0C6AD8A00C0612000CC012F00DC05E
:1094E80013F012501310D8B4090C12C0D9FF13C0CE
:1094F800DAFFDE50DE10D8B4090C12C0D9FF13C051
:10950800DAFFDECF0EF0DDCF0FF00EC0D9FF0FC0AF
:10951800DAFFDF50D8B4090C20EE02F01250D92639
:109528001350DA2212C0E1FF13C0E2FF00EE06F08A
:10953800E650E926E550EA22DE50EE1813E1DE5047
:10954800EE18D8A4090C12C0D9FF13C0DAFF10EE28
:1095580001F0DE50E126DD50E222E75023EC53F023
:109568000E6E0EB0090C000C24EE04F0DE50DE1076
:10957800FBE000C413F001C414F0060E1324D96EE6
:10958800040E1420DA6EDF50116E060E1324D96E05
:10959800060E1420DA6EDF50126E134A142A0D6874
:1095A800010E0E6E13C00FF014C010F00D500F1600
:1095B8000E5010160FC000F410C001F4F29E24EEF5
:1095C80004F0DE06000EDD5AF28E0BC0D9FF0CC087
:1095D800DAFF12C0DFFF24EE04F0010EDBBE05D077
:1095E800000EDE5C020EDE5802E289B29382115050
:1095F80012000E5002E00E5003E10C50D3EF52F06F
:109608000E50D96EDA6A040ED926DE50DE1014E048
:109618000E50D96EDA6A040ED9260E50E16EE26A4F
:10962800020EE126DE50E65CE650800A136EDE503C
:10963800800A1358D8B012000E50D96EDA6A020E9A
:10964800D926DECF0FF0DDCF10F00E50D96EDA6AD2
:10965800DECF11F0DDCF12F00F501124D96E10506B
:109668001220DA6E0CC0DFFF0E50D96EDA6A020ED5
:10967800D926DE2A000EDD22000C0B500F02F3CF94
:1096880013F0F4CF14F0156A166A0B501002F35059
:109698001426F4501522000E16220C500F02F35017
:1096A8001426F4501522000E16220B501102F35006
:1096B8001526F45016220C501002F3501526F450BB
:1096C80016220D500F02F3501526F4501622125090
:1096D8000B02F35016260C501102F35016260D50AB
:1096E8001002F35016260E500F02F350162613C020
:1096F8000BF014C00CF015C00DF016C00EF01200DF
:109708000B0E116E620EE82EFED7112EFCD700D07C
:1097180020D00B0E116E620EE82EFED7112EFCD74C
:1097280000D0010E0B6E0FC0F6FF10C0F7FF000E41
:10973800F86E0F0EF76403D00800F55005D0F6CF89
:10974800E9FFF7CFEAFFEF5099EC4FF00F4A102AE4
:10975800D7D70FC0F6FF10C0F7FF000EF86E0F0E38
:10976800F76403D00800F55005D0F6CFE9FFF7CF2E
:10977800EAFFEF500009CDE11200136A146A156A76
:10978800166A0F5010101110121029E0010E176EF2
:1097980006D0D8900F36103611361236172A12AE68
:1097A800F8D7D89013361436153616360F500B5C8A
:1097B80010500C5811500D5812500E5809E30F5004
:1097C8000B5E10500C5A11500D5A12500E5A13803D
:1097D800D8901232113210320F32172EE2D713C03E
:1097E8000BF014C00CF015C00DF016C00EF01200EE
:1097F800716A706A01018E6B8F6B020E9F6F899080
:109808006F6A9E6B736A030E736401D029D073501C
:10981800070D520EF324D96E010EF420DA6EDF6ABA
:109828007350070D510EF324D96E010EF420DA6E31
:10983800DF6A7350070D500EF324D96E010EF42021
:10984800DA6EDF6A7350070D530EF324D96E010EDA
:10985800F420DA6EDE6ADE6ADE6ADD6A732AD3D73E
:10986800736A1200136E0C0E131807E02EEC53F0F7
:10987800BBEC52F0000901E1FF0C135040090DEC5C
:1098880053F010500DEC53F00F500DEC53F00E50F8
:109898000DEC53F00D500DEC53F0010E126E1350F9
:1098A80002E1950E126E080E131802E1870E126E71
:1098B80012500DEC53F00C0E131802E116EC53F095
:1098C8000A0E126E16EC53F0116E11AE02D0122E63
:1098D800F9D7115012009FEC50F0CC0E94EC52F0D6
:1098E800660E94EC52F077EC52F0156E155005E1C7
:1098F8000F6A106A116A126A1200136A146A135006
:10990800150FD96EDA6A77EC52F0DF6E134A142A13
:1099180014BEF5D7145003E1040E135CF0E318509D
:109928001710161003E1060E155CE2E315C00FF0E0
:1099380016C010F017C011F018C012F01200736AA8
:10994800030E736401D029D07350070D520EF3240F
:10995800D96E010EF420DA6EDF6A7350070D510ECE
:10996800F324D96E010EF420DA6EDF6A7350070D06
:10997800500EF324D96E010EF420DA6EDF6A7350AC
:10998800070D530EF324D96E010EF420DA6EDE6A49
:10999800DE6ADE6ADD6A732AD3D7736A89909F6BA1
:1099A8001200FA93340E0B6E0A0E0C6EF50E0D6E45
:1099B800010E0E6E106A050E0F6EDFEC4FF0390EB9
:1099C8000B6E0A0E0C6EA00E0D6E020E0E6E106A55
:1099D800130E0F6EDFEC4FF00101FA834C0E0B6E85
:1099E8000A0E0C6EE80E0D6E010E0E6E106A0D0E4C
:1099F8000F6EDFEC4FF0496A250E486E56EC35F0D5
:109A0800FA93899012000F5010101110121023E0D1
:109A1800010E136E06D0D8900F3610361136123656
:109A2800132A12AEF8D70F500B5C10500C58115077
:109A38000D5812500E5808E30F500B5E10500C5A78
:109A480011500D5A12500E5AD8901232113210324B
:109A58000F32132EE8D70BC00BF00CC00CF00DC062
:109A68000DF00EC00EF012000FD0030E09D0050E37
:109A78000D6E0101846B856B25D0010E01D0020E9D
:109A88000D6E20D00D6A1ED084C10BF085C10CF07C
:109A98000C5007E0020A0BE00F0A0DE02A0A0FE05B
:109AA800F1D70B500A0AE1E01E0AE1E0EBD70B50B0
:109AB800BC0AE5E0E7D70B50AC0ADFE0E3D70B5070
:109AC8000F0AE0E10D5012000B6A0C6A7350140D76
:109AD800070EF324D96E010EF420DA6EDE6ADE6A10
:109AE800DE6ADD6A7350140D130EF324D96E010E6D
:109AF800F420DA6EDF6A7350140D0F0EF324D96E5A
:109B0800010EF420DA6EDE6ADE6ADE6ADD6A0B4A6E
:109B18000C2A0CBEDBD70C5003E1040E0B5CD6E319
:109B280089906B6A1200B3EC3BF0CAC0E5F0CBC079
:109B3800E6F0E551E61105E0E5C0E1F0E6C0E2F047
:109B4800120082B414D07350200D000EF324A36FBA
:109B5800020EF420A46F000EA56F030EA66F010E6F
:109B6800A86FA76BE30EA96FF5EC0AF0E76FE75152
:109B780004E0E7C0E1F0E26B1200E2EC49F0E16BCF
:109B8800E26B1200196A1A6A186A21D029EC53F09C
:109B98000B500C1011E0180E0B6E0C6AB8EC4AF062
:109BA800176E000E7224D96EDA6A030EDA2217C015
:109BB800DFFF722A194A1A2A18AA07D0000E192498
:109BC800156E040E1A20166E120081AC04D01ABE4F
:109BD800DDD71A04DBE319C015F01AC016F012001D
:109BE8000BC012F00CC013F00DC014F00EC015F02D
:109BF800166A176A0F06D8A010060F2802E1102867
:109C080017E012C0D9FF13C0DAFF124A132ADF5037
:109C1800116E14C0D9FF15C0DAFF144A152ADF5097
:109C2800115C166E176AD8A0170616501710E2E0D6
:109C380016C00BF017C00CF01200010E0B6E0C6A68
:109C480092868D828D8400D000D000D000D08D9473
:109C580000D000D000D000D00D6A0E6A80A602D0D5
:109C68000B500C12D8900B368D9000D000D000D03D
:109C780000D08D8000D000D000D000D08D900D4A4B
:109C88000E2A0EBEEBD70E5003E1030E0D5CE6E381
:109C98000C501200070E106ED00E0F6E0CD016EC82
:109CA80053F0116E11280AE1A00E00D0E82EFDD75E
:109CB8000F06D8A010060F501010F1E1FE0E111873
:109CC80001E0000C16EC53F00BC0D9FF0CC0DAFF12
:109CD800DF6E0B4A0C2A0D06D8A00E060D500E108A
:109CE800F1E116EC53F016EC53F0010C8C6A8A6A19
:109CF8009568936801019C6B726A89928994886B54
:109D0800896B09D0000E8825D96E030E8921DA6E79
:109D1800DF6A884B892B89BFF5D78905F3E3886B00
:109D2800896B09D0340E8825D96E0A0E8921DA6E1E
:109D3800DF6A884B892B89BFF5D78905F3E31200C1
:109D48007BEC51F0000901E1000C0F500DEC53F0D1
:109D5800FD0E0F181EE0020E116E106A0DC0D9FF1D
:109D68000EC0DAFFDF500DEC53F00D4A0E2A100634
:109D7800D8A0110610501110F1E116EC53F016ECB2
:109D880053F016EC53F0126E12501F0B050A01E047
:109D9800000C010C15D00CC0F6FF0DC0F7FF000E2B
:109DA800F86E0F0EF76403D00800F55005D0F6CF13
:109DB800E9FFF7CFEAFFEF50E7EC52F00C4A0D2A23
:109DC8000CC0F6FF0DC0F7FF000EF86E0F0EF7641B
:109DD80003D00800F55005D0F6CFE9FFF7CFEAFF2A
:109DE800EF500009D8E112000EC012F00FC013F0B6
:109DF80010C014F011C015F09FEC50F0CC0E94EC8C
:109E080052F0990E94EC52F00C0E94EC52F0166A43
:109E1800176A1650120FD96EDA6ADF5094EC52F0B6
:109E2800164A172A17BEF5D7175002E09FEF50F0D1
:109E3800040E165CEEE39FEF50F0496EB50E4A6EC5
:109E4800FA0E4B6E486A0AD04AC0F6FF4BC0F7FFBD
:109E58004A4A4B2A0800F550F7E1482A4950481861
:109E680007E04AC0F6FF4BC0F7FF0800F550ECE1E9
:109E78009D0E0001806FFE0E816F49C082F0836BDA
:109E88004AC084F04BC085F0DDEF52F00BC010F0F3
:109E98000CC011F011D00E06D8A00F060D2A0D0423
:109EA800D96EDA6A10C0E1FF11C0E2FF104A112A28
:109EB800DFCFE7FFE7500BE00E500F1008E0EBD7BD
:109EC80010C0D9FF11C0DAFFDF6A104A112A0E0646
:109ED800D8A00F060E28F4E10F28F2E112008980BD
:109EE8000101FA832AEE34F09EC1DFFF000EE8CFAD
:109EF80035FA0D0EE8CF36FA000EE8CF37FA82A40D
:109F080003D0600EE8CF37FA82A406D036CA4EF0E6
:109F1800200E4E124EC036FA496A040E486E56ECB0
:109F280035F0FA939E6B899012000C6E8D9200D0DA
:109F380000D000D000D00BB002D08D9401D08D8419
:109F4800000E0E6E010E0D6E0CAE02D0898A01D085
:109F5800899AD8900C368D908D808D900D4A0E2A56
:109F68000EBEF2D70E5003E1090E0D5CEDE38D82B3
:109F780012009F0E136E146811C015F012C016F06F
:109F88001350152614501622165005E11A0E155CAA
:109F980002E2010E01D0000E176E186A1750181051
:109FA80005E05F0E1114116E126A120011C011F053
:109FB80012C012F012000DC014F00EC015F00BC044
:109FC80012F00CC013F010D014C0D9FF15C0DAFF7E
:109FD800DF50116E144A152A12C0D9FF13C0DAFFD8
:109FE80011C0DFFF124A132A0F06D8A010060F2847
:109FF800EBE11028E9E1120020EE1AF00B50D92607
:10A008000C50DA220DC0DFFF20EE1BF00B50D926D2
:10A018000C50DA220EC0DFFF20EE14F00B50D926C8
:10A028000C50DA220FC0DFFF20EE15F00B50D926B6
:10A038000C50DA221050DF6E12000BC00DF00CC06D
:10A048000EF002D00B4A0C2A0BC0F6FF0CC0F7FF2B
:10A05800000EF86E0F0EF76403D00800F55005D017
:10A06800F6CFE9FFF7CFEAFFEF500009EBE10D501B
:10A078000B5C0B6E0E500C580C6E120089807350DE
:10A08800200D000EF324626E020EF420636E340E6F
:10A09800646E0A0E656E010E676E666AAE0E686EB5
:10A0A800696A4DEC11F00101FA93AEC048F0AFC0F7
:10A0B80049F056EC35F09F6B899012000BC011F0F7
:10A0C8000CC012F00DC013F00EC014F00ED013C067
:10A0D800D9FF14C0DAFF11C0E1FF12C0E2FFDFCFE1
:10A0E800E7FF134A142A114A122A0F06D8A01006AD
:10A0F8000F28EDE11028EBE112000B6E0B500EE07B
:10A1080035EC53F0200EE82EFED738EC53F0CC0E89
:10A1180000D0E82EFDD700D000D0120035EC53F067
:10A12800C00E00D0E82EFDD738EC53F0350EE82EDF
:10A13800FED700F0120035EC53F00A0E0C6EF80E44
:10A14800E82EFED70C2EFCD700D038EC53F0E00EEA
:10A1580000D0E82EFDD704EC53F00D6E090E0C6EFE
:10A16800840EE82EFED70C2EFCD738EC53F00D5099
:10A178001200000EF2BE010E0E6E0C50030BAA6EFA
:10A188000BC0A9FF0DC0A8FFA69EA69CA684F29EA0
:10A19800550EA76EAA0EA76EA682A6B2FED7A694E3
:10A1A8000EB002D0F29E01D0F28E120002D00B4AFD
:10A1B8000C2A0BC0F6FF0CC0F7FF0800F55009E0A9
:10A1C8000BC0F6FF0CC0F7FF0800F5500D180E1075
:10A1D800EEE10BC0F6FF0CC0F7FF0800F5500B6E60
:10A1E8000C6A12005E0E626E5AC063F05BC064F0C7
:10A1F800656A666A676A686A630E546E5CC055F081
:10A208005DC056F0620E576E51EC1FF065505A242F
:10A21800D96E66505B20DA6EDF6A000C186E18AED5
:10A228000ED0189E0D6A0E6A0F6A106A370E36EC49
:10A238004CF0196E010E196402D01950120014C0A6
:10A248000DF015C00EF016C00FF017C010F0185022
:10A2580036EF4CF0010E116E200E0B180C1011E0A9
:10A26800F70E0D6E0E680BC00FF00CC010F00D50FD
:10A278000F260E501022105003E1050E0F5C01E36B
:10A28800116A11C00BF00C6A12005BC04EF05CC082
:10A298004FF04DEC34F05D6E5D500FE15BC00CF09B
:10A2A8005CC00DF071EC4AF05D6E5D5006E15BC07C
:10A2B800D9FF5CC0DAFFDE6ADD6A5D5012009F0ECE
:10A2C8000D6E0E68200E0B100F6E000E0C10106E27
:10A2D8000D500F260E501022105005E11A0E0F5C7B
:10A2E80002E2010E01D0000E0B6E0C6A1200130E72
:10A2F8000C6E880E0B6E0BD016EC53F0FF0A0AE0BA
:10A30800A00E00D0E82EFDD70B06D8A00C060B50E7
:10A318000C10F2E10B500C10D8A4010C000C186AB8
:10A32800196A09D017C00CF00D6A16C00EF0FDECC2
:10A338004AF0184A192A18501424D96E19501520B1
:10A34800DA6EDF50176E1750EDE11200340E0B6E07
:10A358000A0E0C6E0E6A0D6A010E106E0F6A19EC69
:10A3680041F02AEE34F09FC1DFFF496A010E486EC2
:10A3780056EC35F09F6B1200340E0B6E0A0E0C6E05
:10A388000E6A0D6A010E106E0F6A19EC41F0010E8B
:10A39800E8CF34FA0101FA83496A486E56EC35F081
:10A3A800FA9312009F0E0D6E0E680BC00FF00CC0D2
:10A3B80010F00D500F260E501022105005E11A0E05
:10A3C8000F5C02E2010E01D0000E0B6E0C6A120047
:10A3D800BF0E0D6E0E680BC00FF00CC010F00D50C4
:10A3E8000F260E501022105005E11A0E0F5C02E2E3
:10A3F800010E01D0000E0B6E0C6A1200D00E0D6E0D
:10A408000E680BC00FF00CC010F00D500F260E5048
:10A418001022105005E10A0E0F5C02E2010E01D075
:10A42800000E0B6E0C6A1200B886AC84B898440E05
:10A43800AF6EB06AAC98AB8EAB88AB9A9D989D9A7C
:10A44800D08E9F8AF28EAC90AB9CAC9AAC8A9491D9
:10A4580012000BC011F00CC012F008D011C0D9FFC7
:10A4680012C0DAFF0DC0DFFF114A122A0F06D8A06A
:10A4780010060F28F3E11028F1E1120035EC53F033
:10A48800200EE82EFED738EC53F0300EE82EFED71B
:10A4980004EC53F00C6EB00E00D0E82EFDD70C5033
:10A4A8001200106A100E0F6E05D0010E0B6E200EF2
:10A4B80099EC4FF00F06D8A010060F28F6E11028E7
:10A4C800F4E112008450070B0B6E928A80AA02D026
:10A4D800080E0B26020E0101981903E10B1C0F0B45
:10A4E8000B6E0B5012000D6A0E6AD8900D3242ECBA
:10A4F80052F0000901E00D8E0E2A070E0E64F5D702
:10A508000D501200000EE8CF00F4E8CF01F4E8CFB8
:10A5180002F4E8CF03F4E8CF04F4E8CF05F4000C24
:10A528000C6E0D6A0C50010B81EC50F0D8900C3277
:10A538000D2A070E0D64F6D7070C0B6E0B5007E0BB
:10A54800C66A010EC66E400EC76EC68A400CC66A41
:10A55800020EF8D7C2900F0EC16E070EB46E4F0EE2
:10A56800C86E946A948894829482826A12003DEC40
:10A5780053F016EC53F07BEC51F0000901E0010CAC
:10A588002EEC53F0000C0C50030BAA6E0BC0A9FF65
:10A59800A69EA69CA68000F000F0A85012000B6EA4
:10A5A80003D03FEC53F004009EA8FBD70BC0ADFFCF
:10A5B8001200820E476E80C018F081C019F0470E55
:10A5C8001A6E43EF23F00B6E03D03FEC53F00400F8
:10A5D8009EA8FBD70BC0ADFF1200E70000000000EB
:10A5E8000000000000099F02800102E8050109122D
:10A5F80020010001001700002D119420D00F000148
:10A60800928880A803D0010E0B6E01D00B6A0B5004
:10A6180012000B6E0BC0C9FFC7B0FED7C7A0FED78C
:10A62800C9501200C968C7B0FED7C7A0FED7C95025
:10A6380012008980010E6B6E6B6A899012000B6E96
:10A648000B5001E0010C7450120004C40BF005C457
:10A658000CF012003BEC53F016EF53F089909F6B0F
:10A668001200899892981200899892881200828024
:09A6780012008290120012000190
:10FAB400004F4B004449534B5F455252004E4F5444
:10FAC4005F5245414459004E4F5F46494C45004EF4
:10FAD4004F545F4F50454E4544004E4F545F454E82
:10FAE40041424C4544004E4F5F46494C455F535993
:10FAF4005354454D00000D0A202532582025325814
:10FB04002025327320253273202532732025327349
:10FB14002025327320253273202532732025327339
:10FB24002025347320253473202534732025347321
:10FB34002025347320253473202534732025347311
:10FB440020000D0A48504469736B204D6B204949CD
:10FB54002028313846343632302920257320257345
:10FB6400202573205374617274696E672E2E2E0DD6
:10FB74000A000D0A547269656420746F2074616C04
:10FB84006B207768696C7374206E6F742061646491
:10FB9400726573736564000D0A4D61782056656360
:10FBA400746F72206469736B20256420256C642053
:10FBB40028256C582920000D0A253032582530326A
:10FBC400582053533830783A5374617475735B25F5
:10FBD400645D20255820000D0A556E697420256443
:10FBE4002C5365656B20746F20256C6420666169F5
:10FBF4006C6564202564000D0A44736B73656C2086
:10FC040069732025642C206E756D6265722069739A
:10FC14002025642000466F756E6420616E20525466
:10FC2400432066696C652061742025580D0A004CD8
:10FC34006F6F6B696E6720666F7220616E2052541D
:10FC4400432066696C650D0A0046696E6446696CFA
:10FC540065206661696C6564207365617263680D13
:10FC64000A000D0A4469736B2073656C6563742024
:10FC74006E756D626572202564000D0A5365656BAF
:10FC840020746F20256C64206661696C656420258E
:10FC940064000D0A4F70656E696E6720657869733C
:10FCA40074696E6720257320000D0A476F74202540
:10FCB4006C7520202D20726573657474696E6700FD
:10FCC4005365656B696E6720746F20736563746F29
:10FCD400722025580D0A0046696E6446696C6520D9
:10FCE4006661696C656420726561640D0A000D0AC1
:10FCF4004469736B205374617475733A2025582CCE
:10FD040020000D0A57616974696E6720666F72205E
:10FD14006361726420000D0A46696C6520257320B6
:10FD24006973206F70656E20000D0A57726F7465D9
:10FD3400206469736B6E6F3A202564000D0A4F705E
:10FD4400656E696E67206E657720257320000D0A45
:10FD5400545844415441206C656E20256420000DA4
:10FD64000A46696C65202558206973202573200094
:10FD74000D0A4469736B202558206973202573206C
:10FD8400004E6F742061204C4946206469736B0DEA
:10FD94000A000D0A2530325825303258204578693A
:10FDA4007420000D0A52656164696E6720525443E1
:10FDB4000D0A000D0A416D69676F203931323144F3
:10FDC4000D0A000D0A53532F383020393132324492
:10FDD4000D0A000D0A44736B73656C20697320254A
:10FDE4006420000D0A5265616420256420627974E0
:10FDF4006573000D0A487374206279746573322048
:10FE04002564000D0A5772697465206661696C2067
:10FE14002564000D0A4F70656E696E672025732096
:10FE240020000D0A446562756720697320256420EB
:10FE3400000D0A50726F746F2069732025642000CE
:10FE44000D0A5265616420636F6E66696720000D58
:10FE54000A46696C656E616D6520257320005665E0
:10FE640063746F722069732025580D0A0020415471
:10FE74004E2061737365727465642000222A2B2CF2
:10FE84003A3B3C3D3E3F5B5D7C7F000D0A56616C16
:10FE940075653A2025580D0A0072633D2575204684
:10FEA400525F25730D0A000D0A466F726D617474FA
:10FEB400696E6720000D0A4E6F206361726420250D
:10FEC40064002F6C6966646174612E62696E000D52
:10FED4000A25732025582025580D0A000D0A4D6F58
:10FEE400756E74696E6720004D6172203232203263
:10FEF400303230000D0A7362797465732025640012
:10FF04004C6F6164696E672E2E2E0068706469738D
:10FF14006B2E636667005B535251206F66665D000B
:10FF2400466D742065786974200031303A32333A72
:10FF34003437005B2532582025645D005B535251F1
:10FF4400206F6E5D0048504469736B20004E6F2033
:10FF540063617264002D3E2025582000545844618A
:10FF640074610044534B53454C004E414D45255854
:10FF7400004449534B25580072633D256420005BBF
:10FF84004D4C415D0044454255470050524F544F3B
:10FF9400005265616479002025303258007B455257
:10FFA400527D00302E3130004946432000454F49F0
:10FFB400200052454E200041544E200053525120FF
:10FFC4000044415620004E444143004E52464400F2
:10FFD400525443002025580025325800207C20002C
:10FFE400443000443100443200443300443400447B
:0CFFF4003500443600443700256300004F
:020000040020DA
:08000000FFFFFFFFFFFFFFFF00
:020000040030CA
:0E000000FF06191EFF8181FF0FC00FE00F40A9
:00000001FF
